:10274500616D706C20256600506C6561736520694C
:102755006E73657274206D6F64756C6500274C45EA
:10276500442050756C7365722720283078303229E3
:1027750020002020202020696E746F20706F7274F5
:1027850020256264202020200020202020202020D9
:102795002020202020202020202020202000202054
:1027A5002744494E203556272028307832302920B5
:1027B50020200020202020696E746F20706F7274B5
:1027C500203520202020200020002A2A2000202A31
:1027D5002A00202020416464726573733A20202505
:1027E50030345820202020002020526576697369F6
:1027F5006F6E3A202025730057726F6E6720435025
:102805004C44206669726D7761726500536C617620
:102815006520616464723A20256264005265713AEC
:1028250020253032626420213D204163743A202501
:1028350030326264004F76657263757272656E74CC
:10284500203E312E3541206F6E0020202032345637
:10285500206F75747075742021212120202000209F
:102865002020536C61766520616464723A2025628C
:1028750064005245534554004F7665726375727214
:10288500656E74203E302E3541206F6E002020206D
:10289500203556206F757470757420212121002014
:1028A500202020536C61766520616464723A20258E
:1028B5006264002020202055203D2025312E3266DF
:1028C50020560045787465726E616C205472696794
:1028D500676572004672657175656E63793A202584
:1028E500642000487A202020006B487A20202000B0
:1028F5004D487A20202000416D706C6974756465BF
:102905003A2025626420252520202000202D2048FE
:102915007A202B20202020202D20416D70202B0097
:102925004C45442050554C534552002449643A20A7
:102935007363735F323030302E6320323837342082
:10294500323030352D31312D31352030383A34376C
:102955003A31345A2072697474202400013400001D
:102965000046726571000000000101990041900068
:10297500003F80000000000000000000013400005E
:1029850000505769647468000001019A0141A00074
:10299500003F80000000000000000000045D000012
:1029A50001416D706C3030000001019B0042C80090
:1029B500003F80000000000000000000045D0000F2
:1029C50001416D706C3031000001019F0042C8006B
:1029D500003F80000000000000000000045D0000D2
:1029E50001416D706C303200000101A30042C80046
:1029F500003F80000000000000000000045D0000B2
:102A050001416D706C303300000101A70042C80020
:102A1500003F80000000000000000000045D000091
:102A250001416D706C303400000101AB0042C800FB
:102A3500003F80000000000000000000045D000071
:102A450001416D706C303500000101AF0042C800D6
:102A5500003F80000000000000000000045D000051
:102A650001416D706C303600000101B30042C800B1
:102A7500003F80000000000000000000045D000031
:102A850001416D706C303700000101B70042C8008C
:102A9500003F80000000000000000000045D000011
:102AA50001416D706C303800000101BB0042C80067
:102AB500003F80000000000000000000045D0000F1
:102AC50001416D706C303900000101BF0042C80042
:102AD500003F80000000000000000000045D0000D1
:102AE50001416D706C313000000101C30042C80026
:102AF500003F80000000000000000000045D0000B1
:102B050001416D706C313100000101C70042C80000
:102B1500003F80000000000000000000045D000090
:102B250001416D706C313200000101CB0042C800DB
:102B3500003F80000000000000000000045D000070
:102B450001416D706C313300000101CF0042C800B6
:102B5500003F80000000000000000000045D000050
:102B650001416D706C313400000101D30042C80091
:102B7500003F80000000000000000000045D000030
:102B850001416D706C313500000101D70042C8006C
:102B9500003F80000000000000000000045D000010
:102BA50001416D706C313600000101DB0042C80047
:102BB500003F80000000000000000000045D0000F0
:102BC50001416D706C313700000101DF0042C80022
:102BD500003F80000000000000000000045D0000D0
:102BE50001416D706C313800000101E30042C800FD
:102BF500003F80000000000000000000045D0000B0
:102C050001416D706C313900000101E70042C800D7
:102C1500003F80000000000000000000045D00008F
:102C250001416D706C323000000101EB0042C800BB
:102C3500003F80000000000000000000045D00006F
:102C450001416D706C323100000101EF0042C80096
:102C5500003F80000000000000000000045D00004F
:102C650001416D706C323200000101F30042C80071
:102C7500003F80000000000000000000045D00002F
:102C850001416D706C323300000101F70042C8004C
:102C9500003F80000000000000000000045D00000F
:102CA50001416D706C323400000101FB0042C80027
:102CB500003F80000000000000000000045D0000EF
:102CC50001416D706C323500000101FF0042C80002
:102CD500003F80000000000000000000045D0000CF
:102CE50001416D706C323600000102030042C800DC
:102CF500003F80000000000000000000045D0000AF
:102D050001416D706C323700000102070042C800B6
:102D1500003F80000000000000000000045D00008E
:102D250001416D706C3238000001020B0042C80091
:102D3500003F80000000000000000000045D00006E
:102D450001416D706C3239000001020F0042C8006C
:102D5500003F80000000000000000000045D00004E
:102D650001416D706C333000000102130042C80050
:102D7500003F80000000000000000000045D00002E
:102D850001416D706C333100000102170042C8002B
:102D9500003F80000000000000000000045D00000E
:102DA50001416D706C3332000001021B0042C80006
:102DB500003F80000000000000000000045D0000EE
:102DC50001416D706C3333000001021F0042C800E1
:102DD500003F80000000000000000000045D0000CE
:102DE50001416D706C333400000102230042C800BC
:102DF500003F80000000000000000000045D0000AE
:102E050001416D706C333500000102270042C80096
:102E1500003F80000000000000000000045D00008D
:102E250001416D706C3336000001022B0042C80071
:102E3500003F80000000000000000000045D00006D
:102E450001416D706C3337000001022F0042C8004C
:102E5500003F80000000000000000000045D00004D
:102E650001416D706C333800000102330042C80027
:102E7500003F80000000000000000000045D00002D
:102E850001416D706C333900000102370042C80002
:102E9500003F80000000000000000000000000006E
:102EA500000000000000000000000000000000001D
:102EB500000000000000000000000000000000000D
:102EC50000000005F5E10000010002FAF0800002B3
:102ED5000001312D0000050000989680000A0000D1
:102EE5004C4B40001400001E8480003200000F424D
:102EF500400064000007A12000C80000030D400148
:102F0500F400000186A00001010000C35000020189
:102F150000004E2000050100002710000A010000F6
:102F25001388001401000007D0003201000003E8F7
:102F3500006401000001F400C801000000C801F4AC
:0F2F450001000000640001020000000000000015
:1068D7000177010318FF2961C111C10CC112C1134E
:1068E70041019800C10DC10EC10FC11044019000B4
:1068F70000000044019400000000410164FF4101D1
:0869070065FF01750001760037
:024595008F4451
:1045970075840F75A4F575A5FF75A6FF75A70FE4BC
:1045A700F584F5BA75BC9875E880F5D1F58475D1B1
:1045B70003F58475D48075840175D4801271727D7A
:1045C700017F00126E5A7D007F01126E5AE4FF12BE
:1045D7005B52E4FDFF1270C67BFF7A277945900195
:1045E7009BE0FCA3E0FDA3E0FEA3E0F54C8E4B8D22
:1045F7004A8C49122FB6E54460187E007FA27D00E1
:104607007B017A0179991215629001997407F0A3D9
:1046170014F0E4F545E545C37882965009AF451295
:104627006F57054580EFE4F5457B02AD45E4FF1282
:104637006D24EF7033FDFF1270C67BFF7A27794D2B
:10464700122FB67BFF7A277962122FB67BFF7A2764
:104657007977854549122FB67BFF7A27798E122FF6
:10466700B67F00126E8780F90545E545C39405407E
:10467700B87B207D05E4FF126D24EF7030FDFF123B
:1046870070C67BFF7A27794D122FB67BFF7A277981
:10469700A3122FB67BFF7A2779B8122FB67BFF7A42
:1046A70027798E122FB67F00126E8780F9E4F545C1
:1046B700E4F549F54AF54BF54CAB45FD7F01124949
:1046C700090545E545C3940540E6E4FDFF1270C6BC
:1046D700E4F5457B007A00799312000EEEC313FED2
:1046E700EF13FFC374079FFFE49EFEC3E5459FE4F6
:1046F7009E500D7BFF7A2779CD126EDE054580D35C
:104707007BFF7A2779CF126EDE7B007A00799312CE
:104717006EDE7BFF7A2779D3126EDE7D01E4FF120E
:1047270070C67BFF7A2779D7788DE6F54908E6F5D5
:104737004A122FB67D02E4FF1270C67549FF754A0B
:1047470029754B40754C00754D067B017A0279DD62
:10475700126A307B017A0279DD7D20127017E4122C
:104767001234754901754A02754BDD7BFF7A27794B
:04477700ED022FB66A
:10688000E4F58420110FD211F58475D103F5BA75A2
:0D689000BC9875E880C374079F5407F5BBE2
:0D689D0075410275421300D542FCD541F64D
:1068AA00C2AFC2EDD2EC30EDFDD2AFAFBFEFFFAD5C
:1068BA00BEED9002F3CFF0A3EFF0C3E094E89002AC
:0C68CA00F3E0940350047F0180027F0083
:0168D600229F
:103C8800E49002ECF01270EDC8ECC8C9EDC9CAEEB8
:103C9800CACBEFCB900160E0FCA3E0FDA3E0FEA35C
:103CA800E0240AFFE43EFEE43DFDE43CFCD31213AD
:103CB800C4501A1270ED900160E0F8A3E0F9A3E097
:103CC800FAA3E0FBD31213C45003023F281270ED8D
:103CD8009001601214BFE49002EDF09002EDE0FF55
:103CE800C394014003023F377B017A0279EBE4FD7C
:103CF8001260499002EBE0C4540F640260617A00DC
:103D08007B647D017F01125E9820134B127159E488
:103D1800FDFF1270C67BFF7A2779FD126EDE7D01EA
:103D2800E4FF1270C69002EDE0FFD39400400B7BD5
:103D3800FF7A2879118F49122FB67D02E4FF12709D
:103D4800C67BFF7A2879217549029002EBE0FFC40F
:103D5800540FF54A122FB6D2139002EC7401F0906A
:103D680002EDE0FF7544017545027546EE7547039F
:103D7800E4FB7D01124E639002EEE020E303023E75
:103D88000A7A007B647D017F01125E9820124E1230
:103D98007159E4FDFF1270C67BFF7A28793A122F19
:103DA800B67D01E4FF1270C67BFF7A28794F122F87
:103DB800B67D02E4FF1270C69002EDE0FFD39400D6
:103DC800400B7BFF7A2879648F49122FB67D037FD9
:103DD8000F1270C67BFF7A287977122FB6D2127F1E
:103DE80003126880EF60159002EDE0FF126FDCC2ED
:103DF800127F03126880EF70F81271599002EC7408
:103E080001F01270EDE47B64FAF9F8C31213C440B0
:103E180003023F1F9002EDE0FF75440175450275EE
:103E280046F17547027B037D02124E639002F1E072
:103E3800C4F854F0C868FCA3E0C4540F48FDE41269
:103E48000E9CE4FBFA79C87840120C78E4FBFA7906
:103E5800807845120D81E4FBFA79907840120E1EA5
:103E680060025003023F0B200C491271597A007B03
:103E7800647D017F01125E98E4FDFF1270C67BFF2E
:103E88007A28797D122FB67D01E4FF1270C67BFF78
:103E98007A287992122FB67D02E4FF1270C690023A
:103EA800EDE0FFD39400400B7BFF7A2879A48F497B
:103EB800122FB67D03E4FF1270C69002F1E0C4F839
:103EC80054F0C868FCA3E0C4540F48FDE4120E9CEB
:103ED800E4FBFA79C87840120C78E4FBFA79807828
:103EE80045120D818F4C8E4B8D4A8C497BFF7A2869
:103EF80079B8122FB6D20C90023B7401F09002EC04
:103F0800F08014300C119002EDE0FF90023BE06F5E
:103F18007005C20C1271599002EDE004F0023CE306
:103F2800201206200C033013069002EC7401F09066
:043F380002ECE0FFB8
:013F3C002262
:106F57001570A870EFF6A870E6FFC3942A5013EFD8
:106F6700C39400400D74662FF582E43401F58374F1
:056F770001F00570228D
:05717F008F397F0022A2
:0F714A001211EEAB3CAA3DA93E1212347F012276
:10418100301403127159123C88EF60037F0022E45E
:10419100FDFF1270C6900199E070087BFF7A2879C3
:1041A100C880627BFF7A2879D9900199E075F00780
:1041B100A424C5F582E4342EF583E493F549740112
:1041C10093F54A122FB6900199E075F007A424C720
:1041D100F582E4342EF583E49370087BFF7A287925
:1041E100E88022900199E075F007A424C7F582E4E4
:1041F100342EF583E4937BFFB401067A2879EE80AF
:10420100047A2879F5122FB67D01E4FF1270C67B7E
:10421100FF7A2879FC900198E0F549122FB67D03C9
:10422100E4FF1270C67BFF7A297911122FB630088C
:104231000F200D0C900199E0D394004003E014F09D
:1042410030090F200E0C900199E0C394135003E044
:1042510004F0300A18200F15900198E0D394004023
:104261000CE014F01270ED9001901214BF300A3A74
:104271001270EDC8ECC8C9EDC9CAEECACBEFCB903C
:104281000190E0FCA3E0FDA3E0FEA3E02446FFE4EF
:104291003EFEE43DFDE43CFCD31213C4400C90010E
:1042A10098E0D394004003E014F0300B182010156F
:1042B100900198E0C39464500CE004F01270ED900A
:1042C10001941214BF300B391270EDC8ECC8C9ED5E
:1042D100C9CAEECACBEFCB900194E0FCA3E0FDA3E9
:1042E100E0FEA3E02446FFE43EFEE43DFDE43CFCA9
:1042F100D31213C4400B900198E094645003E0047E
:10430100F0900165E0FF900199E06F60057F001278
:104311006F57900164E0FF900198E06F604C754029
:1043210002E540C37882965041900198E0FCE41286
:104331000EA1E4FBFA79C87842120D81EEC0E0EFDC
:10434100C0E0E54075F020A4AB18251AF9E5193550
:10435100F0FA90000D12150CD0E0FFD0E0FE12141F
:1043610038AF40126F57054080B7900198E0900137
:1043710064F0900199E0900165F0A208920DA20904
:0C438100920EA20A920FA20B92107F0075
:01438D00220D
:10570F00900166E06022E4F0900199E075F007A443
:10571F0024C1F9742E35F0754AFFF54B894CE4F529
:10572F0049FBFD7F04124909900167E06014E4F022
:10573F00F549754A01754B01754C9AFBFD7F0512B2
:10574F0049099002DD7402F09002DDE0FFC3788218
:10575F0096505C74662FF582E43401F583E0604760
:10576F009002DDE02466F582E43401F583E4F0EF86
:10577F0075F004A42493F9740135F0754A01F54BC3
:10578F00894C9002DDE0FD24FEFFE434FFFEEF784C
:10579F0003CEC313CE13D8F9FBED24FE5407F549FE
:1057AF00E4FD7F021249099002DDE004F080997B4D
:1057BF00007A00793FE4FDFF125FB9E4FF126880C1
:1057CF00EF24FF92087F01126880EF24FF92097F78
:1057DF0002126880EF24FF920A7F03126880EF2481
:0657EF00FF920B0200A670
:104A7100D2B1C2B0C2B2E49002F5F09002F5E0FE0C
:104A8100C39404504BEFA806088002C333D8FC54EA
:104A910008D394004003D38001C392B30000000007
:104AA1000000000000000000000000000000000005
:104AB100D2B0000000000000000000000000000073
:104AC100000000000000C2B09002F5E004F080ABED
:104AD100E49002F5F09002F5E0FFC39403504BED32
:104AE100A807088002C333D8FC5404D394004003C0
:104AF100D38001C392B30000000000000000000059
:104B010000000000000000000000D2B00000000022
:104B11000000000000000000000000000000000094
:104B2100C2B09002F5E004F080ABE49002F5F090A1
:104B310002F5E0FFC39404504BEBA807088002C3C1
:104B410033D8FC5408D394004003D38001C392B3FB
:104B51000000000000000000000000000000000054
:104B610000000000D2B000000000000000000000C2
:104B710000000000000000000000C2B09002F5E05B
:104B810004F080ABD2B20000000000000000000081
:104B910000000000000000000000D2B00000000092
:104BA1000000000000000000000000000000000004
:104BB100C2B0C2B2C2B3E55824FF92B0D2B2C2B100
:104BC10000000000000000000000000000000000E4
:064BD10000000000C2B26A
:014BD70022BB
:06717900E4F558024A7122
:02630700AC03E5
:106309007B03127179E4900313F0EC5480D3940069
:106319004003D38001C392B30000000000000000D5
:10632900000000000000000000000000D2B00000E2
:106339000000000000000000000000000000000054
:106349000000C2B0EC25E0FC900313E004F0E0B4D7
:1063590008B8C2B3D2B2000000000000000000007B
:1063690000000000000000000000D2B000000000A2
:106379000000000000000000000000000000000014
:04638900C2B0C2B22A
:01638D0022ED
:02638E00AC035E
:106390007B02127179E49002E3F0EC5480D3940014
:1063A0004003D38001C392B300000000000000004E
:1063B000000000000000000000000000D2B000005B
:1063C00000000000000000000000000000000000CD
:1063D0000000C2B0EC25E0FC9002E3E004F0E0B481
:1063E00008B8C2B3D2B200000000000000000000F4
:1063F00000000000000000000000D2B0000000001B
:10640000000000000000000000000000000000008C
:04641000C2B0C2B2A2
:016414002265
:065F29008B1B8A1C891D80
:105F2F00E4FB127179D2B200000000000000000003
:105F3F000000000000000000000000D2B0000000D0
:105F4F000000000000000000000000000000000042
:105F5F0000C2B0C2B2E4900311F0000000000000D4
:105F6F000000000000000000000000000000D2B0A0
:105F7F000000000000000000000000000000000012
:105F8F0000000000C2B0900312E025E0FFA2B4E4CD
:105F9F00334FF0900311E004F0E0B408BD9003120A
:0A5FAF00E0AB1BAA1CA91D0212346E
:065FB9008B408A41894281
:105FBF007B01127179D2B2000000000000000000D6
:105FCF000000000000000000000000D2B000000040
:105FDF0000000000000000000000000000000000B2
:105FEF0000C2B0C2B2E49002DEF000000000000078
:105FFF000000000000000000000000000000D2B010
:10600F000000000000000000000000000000000081
:10601F0000000000C2B09002DFE025E0FFA2B4E470
:10602F00334FF09002DEE004F0E0B408BD9002DFE1
:0A603F00E0AB40AA41A9420212346E
:0461F100AB07AF4702
:0261F500AC03F9
:1061F7007B05127179E49002E3F0EC5480D39400AC
:106207004003D38001C392B30000000000000000E8
:10621700000000000000000000000000D2B00000F5
:106227000000000000000000000000000000000067
:106237000000C2B0EC25E0FC9002E3E004F0E0B41B
:1062470008B8C2B3D2B2000000000000000000008E
:1062570000000000000000000000D2B000000000B5
:106267000000000000000000000000000000000027
:04627700C2B0C2B23D
:01627B002200
:066049008B418A428943ED
:10604F007B04127179D2B200000000000000000042
:10605F000000000000000000000000D2B0000000AF
:10606F000000000000000000000000000000000021
:10607F0000C2B0C2B2E49002F3F0000000000000D2
:10608F000000000000000000000000000000D2B07F
:10609F0000000000000000000000000000000000F1
:1060AF0000000000C2B09002F4E025E0FFA2B4E4CB
:1060BF00334FF09002F3E004F0E0B408BD9002F427
:0A60CF00E0AB41AA42A943021234DB
:10704E007B017A0279E7124D229002E7E0D3940099
:08705E0040047F0180027F0065
:017066002207
:064D22008B468A47894818
:104D28007B07127179D2B300000000000000000078
:104D38000000000000000000000000D2B0000000E9
:104D4800000000000000000000000000000000005B
:104D580000C2B0D2B3000000000000000000000054
:104D6800000000000000000000D2B00000000000B9
:104D7800000000000000000000000000000000C269
:104D8800B0C2B300000000000000000000000000F6
:104D980000000000000000D2B00000000000000089
:104DA80000000000000000000000000000C2B0E4A5
:104DB8009002E8F0C2B3000000000000000000000C
:104DC80000000000000000000000D2B00000000059
:104DD80000000000000000000000000000000000CB
:104DE800C2B09002E8E004F0E0B406C830B409AB01
:104DF80046AA47A948E4805FE49002E8F000000072
:104E0800000000000000000000000000000000009A
:104E180000D2B00000000000000000000000000008
:104E280000000000000000C2B09002EAE025E0FFA8
:104E38009002E9E033FEA2B4E433FDEF4DFFEEF05B
:104E4800A3EFF09002E8E004F0E0B410B09002E9BB
:0A4E5800E0AB46AA47A94812123445
:014E6200222D
:106D24009002E4EFF0A3EDF0A3EBF012704EEF70DD
:106D340002FF229002E4E0FFA3E0FD7B017A0279E6
:106D4400E3124D229002E6E0FF9002E3E0B507046F
:066D54007F0180027F00B8
:016D5A002216
:023F3D00AC03D3
:103F3F007B07127179D2B30000000000000000006F
:103F4F000000000000000000000000D2B0000000E0
:103F5F000000000000000000000000000000000052
:103F6F0000C2B0C2B300000000000000000000005B
:103F7F00000000000000000000D2B00000000000B0
:103F8F00000000000000000000000000000000C260
:103F9F00B0C2B300000000000000000000000000ED
:103FAF0000000000000000D2B00000000000000080
:103FBF0000000000000000000000000000C2B0E49C
:103FCF0090030EF0D2B300000000000000000000CC
:103FDF0000000000000000000000D2B00000000050
:103FEF0000000000000000000000000000000000C2
:103FFF00C2B090030EE004F0E0B406C8D2B20000E5
:10400F0000000000000000000000000000000000A1
:10401F000000C2B2D2B30000000000000000000098
:10402F0000000000000000000000D2B000000000FF
:10403F000000000000000000000000000000000071
:10404F00C2B0C2B30000000000000000000000007A
:10405F000000000000000000D2B0000000000000CF
:10406F000000000000000000000000000000C2B0CF
:10407F00D2B30000000000000000000000000000AC
:10408F00000000000000D2B000000000000000009F
:10409F00000000000000000000000000C2B0E4902B
:1040AF00030EF0C2B300000000000000000000008B
:1040BF00000000000000000000D2B000000000006F
:1040CF00000000000000000000000000000000C21F
:1040DF00B090030EE004F0E0B406C8E490030EF0D5
:1040EF00EC5480D394004003D38001C392B30000FB
:1040FF0000000000000000000000000000000000B1
:10410F000000D2B00000000000000000000000001E
:10411F000000000000000000C2B0EC25E0FC90039E
:10412F000EE004F0E0B410B8D2B2000000000000BE
:10413F000000000000000000000000000000C2B2FC
:0A414F00E490030FF0A3F020B42762
:0D415900751E01751F0300D51FFCD51EF655
:10416600900310E004F0700690030FE004F0900353
:0A4176000FE0B427DBA3E0B410D67D
:01418000221C
:10438E0008760008764D1570A870A6491570A870AD
:08439E00A648AB477D027F0237
:1043A6001570A870A6031570A870A6051570A870DC
:0843B600A607E57024F9F5707B
:1043BE002408F8E66402600302458CE570240CF8CC
:1043CE00860308E6FA08E6F91213E8A8701214B389
:1043DE00E5702407F8E6B4020F7F007EFF7D7F7C38
:1043EE0047A87012146A804AE5702407F8E6B48272
:1043FE001DE4FBFA79207840C000A870121452D048
:10440E0000120D817B007AFF797F78478024E5705A
:10441E002407F8E6B4832BE4FBFA79C87841C00090
:10442E00A870121452D000120D817B007AFF797F92
:10443E007847120C78120ED5E5702404F8A60608FB
:10444E00A607E5702409F8E6FFE570240AF8E6FDF4
:10445E007B06127179E5702406F8E4F6E570240601
:10446E00F8E6FFC39404503FEF94014003D380015C
:10447E00C392B30000000000000000000000000026
:10448E0000000000000000D2B0000000000000009C
:10449E0000000000000000000000000000C2B0E5B7
:1044AE00702406F80680B5E5702406F8E4F6E5708B
:1044BE002406F8E6C394045051E570240BF8E6FF89
:1044CE005408D394004003D38001C392B30000007C
:1044DE0000000000000000000000000000000000CE
:1044EE0000D2B0000000000000000000000000003C
:1044FE0000000000000000C2B0E570240BF8EF25AC
:10450E00E0F6E5702406F80680A4E5702406F8E4CB
:10451E00F6E5702406F8E6C394105060E5702404A6
:10452E00F8E6FE08E6FFEE5480FCD3E49400EC942B
:10453E00004003D38001C392B300000000000000CE
:10454E0000000000000000000000000000D2B000DB
:10455E00000000000000000000000000000000004D
:10456E00000000C2B0E5702404F8EF25E0FFEE3342
:10457E00F608A607E5702406F8068095D2B17F01ED
:07458E00E570240FF5702217
:064909008F468D478B482C
:10490F00E5466401702A74062548F582E43403F500
:10491F0083E4F0FBAD48AF4712638EE4F550F54FDB
:10492F00F54EF54D157015701570A870F612438E73
:10493F00E546640260030249C7AB4AAA4BA94C1271
:10494F0013E88F508E4F8D4E8C4D1570157015705E
:10495F00A870760012438EE4FFFEFDFCAB50AA4F09
:10496F00A94EA84D120E1E701F74062548F582E43D
:10497F003403F583E0FFAE497401A806088002C333
:10498F0033D8FCF45FF0801C74062548F582E434BC
:10499F0003F583E0FFAE497401A806088002C33314
:1049AF00D8FC4FF074062548F582E43403F583E014
:1049BF00FBAD48AF4712638EE54664046003024ABD
:1049CF0051AB4AAA4BA94C1213E88F548E538D52F8
:1049DF008C517D031261F1AF54AE53AD52AC51788F
:1049EF00081213D58F548E538D528C517D04126142
:1049FF00F1AF54AE53AD52AC5178081213D58F545A
:104A0F008E538D528C51AB077D05AF471261F5AFB9
:104A1F0054AE53AD52AC5178081213D58F548E53F8
:104A2F008D528C51AB077D06AF471261F5AF54AE77
:104A3F0053AD52AC5178081213D58F548E538D52FB
:104A4F008C51E546B40518AB4AAA4BA94C1211EE8E
:104A5F00FBD3941440027B147D02AF471261F57FA4
:014A6F000145
:014A70002223
:106DC80020202020557067726164696E670020205A
:106DD80020204669726D776172652E2E2E00323042
:106DE80031362D30362D3237202D2064393161323D
:036DF800346600FE
:0F690F000184FF420010FFFF4400180000000049
:104BD8007BFF7A6D79E67D2D1269DAEA494B601917
:104BE8007BFF7A6D79E67D2D1269DAE92402F9E412
:104BF8003A8B44F54589468004E4FEFF22AB44AA7B
:104C080045A946900001121207FFC3648094B04082
:104C18000ED3EF648094B95006EF24D0FF801E9025
:104C28000001121207FFC3648094E1400ED3EF64C1
:104C38008094E65006EF24A9FF80027F00EF7D00F4
:104C4800FC1211EEFFC3648094B0400ED3EF648071
:104C580094B95006EF24D0FF8021AB44AA45A94659
:104C68001211EEFFC3648094E1400ED3EF64809488
:104C7800E65006EF24A9FF80027F00EFC454F04CF1
:104C8800FCAB44AA45A946900002121207FFC36470
:104C98008094B0400ED3EF648094B95006EF24D0CE
:104CA800FF801E900002121207FFC3648094E14047
:104CB8000ED3EF648094E65006EF24A9FF80027FAC
:104CC80000EF75F010A4FFEC45F0FEED4FFF9000EB
:104CD80003121207FDC3648094B0400ED3ED6480C4
:104CE80094B95006ED24D0FD8024AB44AA45A946CA
:104CF800900003121207FDC3648094E1400ED3EDC7
:104D0800648094E65006ED24A9FD80027D00EF4DF5
:094D1800FF9002DDEEF0A3EFF0C4
:014D2100226F
:1036F100E47880F6127113C28575840F75E104E4D4
:10370100F5E275E344F58475B7B075840F758A8366
:10371100F597438901758D01758F01758E04F54209
:10372100F5430543E54370020542640F454270F2DB
:10373100438902E4F542F543AE42AF43E4FCFD7B2D
:10374100507AC3F9F8D31213AE400FE58920E40A89
:103751000543E54370E2054280DE75970212656D0F
:103761001266448F41E4F584E541D39400400EE5AF
:10377100EF5402D394004005AF4112477B126F9E74
:10378100E4FF126FBD43EF04E4F542F5437D01AF61
:1037910043126E5A0543E54370020542C39402E5A4
:1037A10042940040E8E4F520C22AC228C22EC22D6C
:1037B100C22C7880F6C22F08F67886F618F6788B38
:1037C100F6F542F54374202543F58274003542F540
:1037D10083E4F00543E54370020542B400E7E542A6
:1037E100B401E2E4F542F54374202543F582740106
:1037F1003542F583E4F00543E54370020542644038
:10380100454270E4E4F584E5EF20E10CE5EF54086E
:10381100D394004003D38001C392037D08E4FF12D7
:103821006AD37D087F01126AD3E4788AF67882F63A
:10383100AB18AA19A91A7882E6FF75F020A4F582BF
:1038410085F083121207FE788A26F6EE60057882EB
:103851000680DDEFD394004032AB18AA19A91A9063
:10386100000D12150C1211EEF5417455121234129D
:1038710011EE64556002D22C74AA1212341211EEA8
:1038810064AA6002D22CE541121234E4F584E5EF1A
:103891005402D3940040047F018002E4FF125627B2
:1038A1008F40E54020E036C22974FF788DF608F696
:1038B10008F608F67E007F107D007B007A00799380
:1038C1001215627549FF754A29754B25754C0075AE
:1038D1004D107B007A007993126A308002D229124E
:1038E1004BD87891A60608A607E54030E1030239D6
:1038F10095E4F542F543E543AE427805C333CE3353
:10390100CED8F9FFAB18AA19A91AF5828E83121223
:10391100076078E92FF9EA3EFA90000412120720B5
:10392100E25EE4F53FE53FC37877965053E543AE59
:10393100427805C333CE33CED8F9AB18AA19A91AE8
:10394100F5828E83121207FF7E00C006C0077D003C
:10395100E543AE427805C333CE33CED8F929F9EA2F
:103961003EFA90000D12150C788AE6853FF0A429E5
:10397100F9EA35F0FAD007D006121562053F80A5A5
:103981000543E543700205420238F77F0112459570
:10399100C22B8007E4FF124595D22BE4F542F54393
:1039A1007A007B967D03AF43125E980543E5437031
:0C39B100020542C39402E542940040E489
:0139BD0022E7
:05718400788BE6FF22FC
:0300230002520284
:10520200C0E0C0F0C083C082C0D075D000C000C072
:1052120001C002C003C004C005C006C00730993EE9
:10522200C2997886067986E77881667015F678865F
:01523200F685
:0D52330075270A75281300D528FCD527F62D
:04524000C285801C87
:0D52440075271475281300D528FCD527F612
:105251007886E62420F582E43401F583E0F599208F
:1052610098030252FD209A08202A05C2980252F999
:10527100C29A7885E6062420F582E43400F583E5B8
:1052810099F0C298E6FFB40112900020E0FE70038D
:10529100F68069EE54072402788CF6EFB4020D789B
:1052A1008CE6B40907900021E02403F67885E6FF37
:1052B100B40007E4B40103F68042EFC3788C964052
:1052C1003B7885E624FFFDE434FFFC7B017A00791D
:1052D100201260D97885E6241FF582E43400F58335
:0852E100E06F60047600801408
:0D52E90075271475281300D528FCD527F66D
:1052F60012161078857600D007D006D005D004D0D7
:1053060003D002D001D000D0D0D082D083D0F0D04C
:02531600E03283
:10002600900021E075F020A4AB18251AF9E51935E2
:10003600F0FA90000D12150C788BE6FF18E68FF09B
:10004600A4252BF582E435F0F583121207FF7B0019
:040056007A0079298A
:10005A008F398B3A8A3B893CE4F584EA494B601C28
:10006A00AB3AAA3BA93C1211EEFFE539FD7C00121E
:0C007A007166AB3AAA3BA93CEF121234AD
:0D008600753D14753E1300D53EFCD53DF6CA
:0E0093008539997F01126E873099FDC299223E
:106D92009001207478F07885E6241FF582E43400AF
:096DA200F583E0900121F07F026D
:096DAB00E4F5847881EFF6D2854D
:0D6DB400753914753A1300D53AFCD539F63F
:076DC100900120E0F599228A
:106C5900C9EFC9E964017028EDC39B40347877E630
:106C6900FFEB2FFFE433FEEDC39FEE6480F87480E1
:106C790098501ED22AC3ED9B788BF678877601222D
:106C8900B90214ED6B700AD22A788BF678877602EE
:086C990022C22AE47887F622EA
:10671700C9EFC9BAFF15BBFF12ED6B7002EC6A70C7
:1067270049D22A788BF67887E9F622E96401702541
:10673700C3ED9BEC9A401C7877E62BFFE43AFEC347
:10674700ED9FEC9E500DD22AC3ED9B788BF6788790
:106757007601228015B90218ED6B7002EC6A700A97
:10676700D22A788BF67887760222C22AE47887F6CF
:0167770022FF
:10161000900020E0FF54F8F52AE4F584EF12153C21
:10162000166009166D0A168010168911169A121680
:10163000B11916C71A16EC2016F528179129189318
:101640003318CE3718FE39191841192349192E4E6F
:1016500019615019A961185D7019A198000019D974
:10166000900021E0FD788EE6FB7F0180279000212D
:10167000E0FCA3E0FD788DE6FA08E6FB7F01802B15
:10168000D22A788776030219D9900021E0FD78905C
:10169000E6FB7F02126C590219D9900021E0FCA3ED
:1016A000E0FD788FE6FA08E6FB7F02126717021961
:1016B000D9900021E0FD788EE6FB7F01126C592065
:1016C0002A030219D9801A900021E0FCA3E0FD78DA
:1016D0008DE6FA08E6FB7F01126717202A0302193C
:1016E000D99001207478F07F010219D6E4F5847551
:1016F000EF100219D9C2ACE4F529D285FB7A007942
:10170000297F7F12005A7B007A0079297F1E120000
:101710005A7B007A0079297F0512005A7882E612F6
:101720000053788DE6120053788EE6120053788FBE
:10173000E61200537890E61200537891E6120053B7
:101740007892E6120053E4F52B7493252BF8E612F9
:101750000053052BE52BC3941040EEE4F52B740ADF
:10176000252BF582E43400F583E0120053052BE5C8
:101770002BC3940640E87B007A007900AF29120061
:011780005A0E
:0D17810075370A75381300D538FCD537F6DA
:10178E00021848900021E0FFC378829640030218A9
:10179E004FEF75F020A4251AF9E51935F0851834A8
:1017AE00F5358936C2ACE4F529D285FB7A00792964
:1017BE007F7F12005A7B007A0079297F0D12005A22
:1017CE00AB34AA35A9361211EE120053AB34AA353A
:1017DE00A936900001120050AB34AA35A9369000FC
:1017EE0002120050AB34AA35A936900003120050F5
:1017FE00AB34AA35A936900004120050E4F52BAB99
:10180E0034E5362405F9E43535FA7E00E9252BF961
:10181E00EE3AFA1211EE120053052BE52BC3940883
:0D182E0040DD7B007A007900AF2912005ADE
:0D183B0075370A75381300D538FCD537F61F
:10184800C285D2AC0219D99001207478F0E4A3F0D3
:101858007F020219D612710078A31214B3900120E6
:10186800747CF078A3E6A3F008E6A3F008E6A3F0FA
:1018780008E6A3F07C007D057B017A0179201260DF
:10188800D9900125EFF07F060219D6900021E0FFDC
:10189800B4010FA3E0FDA3E0788DCDF608EDF602C4
:1018A80019A1EFB4020A900022E0788DF60219A17E
:1018B800900021E0B4030CA3E0FFA3E0788FCFF6FB
:1018C80008EFF60219A1E4F52B900021E0FFE52BC3
:1018D800C39F501B7422252BF582E43400F583E066
:1018E800FF7493252BF8EFF6052BE52BB410DAE4FB
:1018F80078A2F60219A17A007B327D01788BE6FF87
:10190800125E98900021E0FDE4FF126AD30219D913
:10191800900021E024FF92020219D9900021E024CE
:10192800FF92010219D97A007B327D017F00125E95
:1019380098E4F52B7421252BF582E43400F583E037
:10194800FF7412252BF582E43400F583EFF0052BA4
:10195800E52BB406DFD22F8078788BE66005752DED
:1019680002800B202D05752D038003752D01900134
:10197800207479F0A3E52DF07C007D027B017A01CB
:1019880079201260D9900122EFF07F03126DABE548
:101998002D6401703CD22E8002D228788076F180A6
:1019A800307A007B327D017F00125E9890012074AE
:1019B80079F0900021E0900121F07C007D027B010C
:1019C8007A0179201260D9900122EFF07F03126D1D
:1019D800ABE52A64A06003021BE8900020E064A144
:1019E8006003021AD8A3E0C37882964003021ACD96
:1019F800AB18AA19A91AE0FF75F020A4F58285F0A2
:101A080083121207F52DEF75F020A429F9EA35F0B5
:101A1800FA90000412120730E237900021E01271A8
:101A28007F8F2D900120747FF0A3E52DF02402FD17
:101A3800E433FC7B017A0179201260D97422252DC8
:101A4800F582E43401F583EFF0E52D2403FF021B52
:101A5800E5900021E0FF12717FC2ACE4F529D28540
:101A6800E52DD39406402B7B007A0079297F7F12DD
:101A7800005A7B007A007929AF2D12005AE4F52B21
:101A8800E52BC3952D5007120026052B80F2052D56
:101A98008018E52D2478120053E4F52BE52BC39527
:101AA8002D5007120026052B80F27B007A00790062
:051AB800AF2912005AE5
:0D1ABD0075370A75381300D538FCD537F69B
:101ACA00021BD79001207478F07F01021BE5900079
:101ADA0020E064A26003021BE87882E6FFA3E0FE2E
:101AEA00C39F4003021BDDA3E0FDC39F4003021B0B
:101AFA00DDEE9D4003021BDD900021E0F52BE4F5AD
:101B0A0032F533900022E0FFE52BD39F5026AF2B0E
:101B1A0012717FAB18AA19A91A75F020E52BA4F542
:101B2A008285F0831212072533F533E43532F53214
:101B3A00052B80CFC2ACE4F529D285FB7A0079293E
:101B4A007F7F12005AC3E5339480E5329400500235
:101B5A008007E5324480120053AF331200549000DC
:101B6A0021E0F52B900022E0FFE52BD39F5046E4BD
:101B7A00F52CAB18AA19A91A75F020E52BA4F58241
:101B8A0085F083121207FFE52CC39F5024E52B75BD
:101B9A00F020A429F9EA35F0FA90000D12150C7814
:101BAA008BE6FF18E68FF0A4252C120049052C803D
:101BBA00C1052B80AF7B007A007900AF2912005A49
:0D1BCA0075370A75381300D538FCD537F68D
:101BD700C285D2AC800B9001207478F07F01126D22
:101BE700ABE52A6458704DFA7B327D01788BE6FFAE
:101BF700125E98753C01753D01753E217B017A00A7
:101C0700792112714A8F2DE52D2478900120F0EF6C
:101C17002401FDE433FC7B017A0179201260D97439
:101C270021252DF582E43401F583EFF0E52D24021B
:101C3700FF126DABE52A64806009E52A64886003BA
:101C4700021DFA7887E6B4010F7A007B327D0178AE
:101C57008BE6FF125E98801AE4F52BE52BC37877A5
:101C670096500F7A007B327D01AF2B125E98052BC1
:101C770080E9900020E05407F52DB4070A752C0180
:101C8700A3E0F52DA38006E4F52C900021E0F52EC6
:101C9700152DE52EC37882964003021DFAAB18AACC
:101CA70019A91A75F020E52EA4F58285F083121282
:101CB70007FFE52DD39F40028F2D7887E6B40109F2
:101CC700788BE6F531F5308009E4F5307877E6145E
:101CD700F531788BA630788BE6D395314003021D1A
:101CE700D1E4F52BE52BC3952D4003021DC6E52E48
:101CF70075F020A4AB18251AF9E51935F0FA90000C
:101D07000412120730E203021DC1900001121207EC
:101D170064387041E52DD394044011E52C252B241C
:101D270022F582E43400F583E0FD80707885E6C310
:101D3700952BFFE49400FE741E2FF58274003EF588
:101D470083E0FDE52E75F020A4AB18251AF9E519F7
:101D570035F0FA8047AB18AA19A91A75F020E52EB5
:101D6700A4F58285F083121207FF7885E6C39FFFEB
:101D7700E49400FE7C00EF252BFFEC3EFEEF252CC4
:101D8700FFEC3EFE741F2FF58274003EF583E0FDE5
:101D9700E52E75F020A429F9EA35F0FA90000D1226
:101DA700150C788BE6FF18E68FF0A4FFE52B2FF5CF
:101DB70082E435F0F583ED121246052B021CEBAFDA
:101DC7002E126F57788B06021CDD788BA630E52E16
:101DD70075F020A4AB18251AF9E51935F0FA90002B
:101DE7000412120730E5047884A62EE52AB4880386
:101DF700126D92E52A64A86003021F327887E6B461
:101E0700010F7A007B327D01788BE6FF125E9880A6
:101E17001AE4F52BE52BC3787796500F7A007B32BF
:101E27007D01AF2B125E98052B80E9900021E030F1
:101E3700E711547FFEA3E0FDEEF532EDF533752C87
:101E470003800C900021E0753200F533752C027485
:101E570020252CF582E43400F583E0FF7421252C3E
:101E6700F582E43400F583E0F52F8F2EE52ED39528
:101E77002F4003021F2FE52EC37882964003021FCF
:101E87002AAB18AA19A91A75F020E52EA4F58285A0
:101E9700F083121207F52D7887E6B40109788BE6EF
:101EA700F531F5308009E4F5307877E614F53178C7
:101EB7008BA630788BE6D39531505EE4F52BE52B76
:101EC700C3952D504AE52E75F020A4AB18251AF9B5
:101ED700E51935F0FA90000412120720E22DE52CDF
:101EE700252B2422F582E43400F583E0FD90000DD4
:101EF70012150C788BE6FF18E68FF0A4FFE52B2F61
:101F0700F582E435F0F583ED121246052B80AFAF6D
:101F17002E126F57788B06809A788BA630E52D2581
:0B1F27002CF52C052E021E73126D928B
:011F3200228C
:09692E0090001D121330FFAEF0C1
:106937008E418F42900010E065417004A3E06542EC
:10694700603A900000740AF0E541A3F0E542A3F035
:106957007C007D037B017A0079001260D9900003E7
:10696700EFF07B017A0079007548017D047C001205
:0D6977005E06900010E541F0A3E542F0221D
:036A8200CCEECC8B
:106A8500900000741AF0A3ECF0EFA3F07C007D03F6
:106A95007B017A0079001260D9900003EFF07B0149
:106AA5007A0079007548017D047C00125E067B0141
:106AB5007A0079007D0A7C00125A90EF7002FF225D
:0D6AC500900000E0647860037F00227F01F4
:016AD20022A1
:106E2D007A007B327D017F01125E9874FF90001015
:106E3D00F0A3F07F0A900000E4F0A3DFFC7B017A61
:0D6E4D000079007548017D0A7C00025E0698
:1050D700E4F53FE53FC37882964003025201E53F7E
:1050E70075F020A4AB18251AF9E51935F0FA9000E8
:1050F7000412120720E4030251FC12692E900000EB
:1051070074A1F0E53F75F020A4AB18251AF9E5194D
:1051170035F0FA90001F121207900001F07C007D15
:10512700027B017A0079001260D9900002EFF07BD0
:10513700017A007900E4F5487D03FC125E067B01E5
:105147007A0079007D647C00125A908F40E540C355
:1051570094025002804DE5402476FF900000E06FF6
:105167006002803FAB18AA19A91A75F020E53FA481
:10517700F58285F083121207FFE54024FE6F600277
:105187008021E54024FFFDE434FFFC7B017A0079B0
:10519700001260D974FF2540F582E434FFF583E0FF
:1051A7006F6007AF3F126E2D804BC2AFAB18AA19C5
:1051B700A91A75F020E53FA4F58285F0831212073E
:1051C700FF7E00EEC0E0EFC0E0E53F75F020A429C8
:1051D700F9EA35F0FA90000D12150CC8E9C8CCEAC7
:1051E700CCCDEBCD7B017A007901D0E0FFD0E0FE9A
:0A51F7001211C8D2AF053F0250DAD2
:01520100228A
:02627C008F3F52
:10627E00EF75F020A4AB18251AF9E51935F0FA12CE
:10628E00692EAB18AA19A91A75F020E53FA4F5825C
:10629E0085F083121207F5402481900000F0E53F4F
:1062AE0075F020A429F9EA35F0FA90001F121207B2
:1062BE00900001F0AF407E0090000D12150C780298
:1062CE007C007D011211C8E5402402FDE433FC7B05
:1062DE00017A0079001260D974022540F582E43407
:1062EE0000F583EFF07B017A007900E5402403FD91
:0962FE00E433FCE4F548025E06FD
:106C10001270EDC8ECC8C9EDC9CAEECACBEFCB9073
:106C20000018E0FCA3E0FDA3E0FEA3E0240AFFE4DB
:106C30003EFEE43DFDE43CFCD31213C4400C125074
:106C4000D71270ED9000181214BF7884E6FFF4603C
:096C50000712627C788476FF22B1
:10F000007880E664F1600302F668E478ADF608F60D
:05F010007881E6601E9E
:0DF01500753F0A75401300D540FCD53FF64D
:10F0220078AE06E61870010678ADB627E108B6108C
:10F03200DDC2AF7584015398FC75FFDE75FFADE448
:10F0420078A9F618F6E4F584209830E478ADF6084D
:10F05200F6209823C378AEE6948818E694135017E6
:0DF06200753F0A75401300D540FCD53FF600
:10F06F0078AE06E61870DD0680DAB28680CD78A815
:10F07F00A699C298E6FF641A6008EF640A6003025B
:10F08F00F168E478ADF608F6209823C378AEE694DD
:07F09F008818E694135017D6
:0DF0A600753F0A75401300D540FCD53FF6BC
:10F0B30078AE06E61870DD0680DA30988778A9A660
:10F0C30099C298E478ADF608F6209823C378AEE6A3
:08F0D300948818E6941350170D
:0DF0DB00753F0A75401300D540FCD53FF687
:10F0E80078AE06E61870DD0680DA20980302F0474D
:10F0F80078A9A699C298E478ADF608F6209823C3B3
:0BF1080078AEE6948818E694135017C8
:0DF11300753F0A75401300D540FCD53FF64E
:10F1200078AE06E61870DD0680DA20980302F04714
:10F1300078A9A699C29818E6641A600302F659D213
:03F1400085C299EC
:0DF14300753F1475401300D540FCD53FF614
:06F150007599783099FD6D
:0DF15600753F0A75401300D540FCD53FF60B
:10F16300C28502F65978A8E6FF6450600302F1FDF8
:10F1730078ADF608F6209823C378AEE6948818E6AF
:04F18300941350177A
:0DF18700753F0A75401300D540FCD53FF6DA
:10F1940078AE06E61870DD0680DA20980302F047A0
:0AF1A40078A9A699C298D285C299F5
:0DF1AE00753F1475401300D540FCD53FF6A9
:08F1BB007599793099FDC299A4
:0DF1C300753F1475401300D540FCD53FF694
:08F1D0007599013099FDC29907
:0DF1D800753F1475401300D540FCD53FF67F
:06F1E500E4F5993099FDEC
:0DF1EB00753F0A75401300D540FCD53FF676
:0EF1F800C28502F659EF6401703ED285C299BD
:0DF20600753F1475401300D540FCD53FF650
:08F213007599783099FDC2994C
:0DF21B00753F1475401300D540FCD53FF63B
:06F22800E4F5993099FDA8
:0DF22E00753F0A75401300D540FCD53FF632
:10F23B00C28502F65978A8E66402600302F30C78E3
:10F24B00ADF608F6209823C378AEE6948818E694BA
:03F25B0013501736
:0DF25E00753F0A75401300D540FCD53FF602
:10F26B0078AE06E61870DD0680DA20980302F047C8
:10F27B0078A9A699C298E408F618E6FF13B392860C
:10F28B00EF25E0FEC3E49400EE94F0502DE6FD7FF5
:10F29B000025E0FEC394E05021ED20E024E4F5844A
:10F2AB0043B701758F0378AFEEF608EFF6F5828E54
:10F2BB0083E4F053B7F0F58F800478AA76FFE4F57A
:05F2CB0084D285C29908
:0DF2D000753F1475401300D540FCD53FF686
:08F2DD007599783099FDC29982
:0DF2E500753F1475401300D540FCD53FF671
:08F2F20078AAE6F5993099FDB8
:0DF2FA00753F0A75401300D540FCD53FF666
:10F30700C28502F65978A8E66403600302F46778B9
:10F31700ADF608F6209823C378AEE6948818E694ED
:03F3270013501769
:0DF32A00753F0A75401300D540FCD53FF635
:10F3370078AE06E61870DD0680DA20980302F047FB
:10F3470078A9A699C298E478ADF608F6209823C361
:0BF3570078AEE6948818E69413501777
:0DF36200753F0A75401300D540FCD53FF6FD
:10F36F0078AE06E61870DD0680DA20980302F047C3
:10F37F0078ABA699C29878A9E6FF139286EF25E09D
:10F38F00FEC3E49400EE94F0400302F047E67D00E4
:10F39F0025E0FCC394E0400302F047E4F58443B753
:10F3AF0001758F0178ABE675F020A42DFFE5F03CD9
:10F3BF0078AFF608EFF6E4F58478ACF678ACE6C3F0
:10F3CF009420504CE408F608F6209823C378AEE654
:08F3DF00948818E694135017FE
:0DF3E700753F0A75401300D540FCD53FF678
:10F3F40078AE06E61870DD0680DA20980302F0473E
:10F4040078AF0806E618CEE6CE70010614F5828EB3
:10F4140083E599F0C29878AC0680ACE4F58453B7E0
:09F42400F0F58FF584D285C29940
:0DF42D00753F1475401300D540FCD53FF627
:08F43A007599783099FDC29923
:0DF44200753F1475401300D540FCD53FF612
:06F44F00E4F5993099FD7F
:0DF45500753F0A75401300D540FCD53FF609
:10F46200C28502F65978A8E6FD6404600302F52419
:10F4720078ADF608F6209823C378AEE6948818E6AD
:04F482009413501778
:0DF48600753F0A75401300D540FCD53FF6D8
:10F4930078AE06E61870DD0680DA20980302F0479E
:10F4A30078A9A699C298E625E078B1F608E4F6783B
:10F4B300AAF678ADF608F678B10806E618CEE6CED9
:10F4C30070010614F5828E83E49378AA26F678AE4B
:10F4D30006E61870010678AEE6700418E66402705A
:05F4E300D6D285C2999C
:0DF4E800753F1475401300D540FCD53FF66C
:08F4F5007599783099FDC29968
:0DF4FD00753F1475401300D540FCD53FF657
:08F50A0078AAE6F5993099FD9D
:0DF51200753F0A75401300D540FCD53FF64B
:10F51F00C28502F659ED6405600302F64D78ADF62B
:10F52F0008F6209823C378AEE6948818E694135013
:01F53F0017B4
:0DF54000753F0A75401300D540FCD53FF61D
:10F54D0078AE06E61870DD0680DA20980302F047E3
:10F55D0078A9A699C298E478ADF608F6209823C349
:0BF56D0078AEE6948818E6941350175F
:0DF57800753F0A75401300D540FCD53FF6E5
:10F5850078AE06E61870DD0680DA20980302F047AB
:0AF5950078ABA699C298D285C299FE
:0DF59F00753F1475401300D540FCD53FF6B4
:08F5AC0075997F3099FDC299A9
:0DF5B400753F1475401300D540FCD53FF69F
:10F5C1007599203099FD78A9E625E0FC78ABE675C0
:10F5D100F020A42400FFE5F03C78B1F608EFF6E452
:08F5E10078AAF678ACF6C29995
:0DF5E900753F1475401300D540FCD53FF66A
:10F5F60078B1E6FE08E6F5828E83E493F5993099B4
:10F60600FD78B10806E618CEE6CE70010614F5823E
:10F616008E83E49378AA26F678AC06E6B420C2C2B6
:01F62600994A
:0DF62700753F1475401300D540FCD53FF62B
:08F6340078AAE6F5993099FD72
:0DF63C00753F0A75401300D540FCD53FF620
:10F64900C285800C78A8E6B40606E4F58475EF1047
:0FF6590078A8E66407600302F0477880F6D2AF26
:01F66800227F
:1057F5007F00126E8720290B7A007B327D017F00A6
:10580500125E98302C0B7A007B1E7D017F00125EA4
:1058150098302817302D147A007B327D01788BE67D
:10582500FF125E98C228125CC8D229202B0C302D9D
:1058350009788076F1125CC8D22B302E2A302D27BC
:10584500C22E127159E4FDFF1270C67BFF7A6D7985
:10585500C8126EDE7D01E4FF1270C67BFF7A6D799A
:10586500D6126EDE12F000302F0B7B017A00791212
:10587500126415C22F1270EDC8ECC8C9EDC9CAEE85
:10588500CACBEFCB90001C12145EEF245AFFE43E06
:10589500FEE43DFDE43CFCD31213C4500F1270ED41
:1058A50090001C121477D31213C440121270ED909D
:1058B500001C1214BF7B017A00790A1259B5202DFC
:1058C500121270EDE47B2C7A01F9F8C31213C4505F
:0458D50002D22D22AC
:10708000E4F58475EF027F64DFFE1236F11257F5E6
:08709000126C1012570F80F57D
:104F9E004D656D6F727920746573742E2E2E004DD3
:104FAE00656D6F7279206572726F722062616E6BC1
:104FBE002025626400005EBCE2613FDD83C29C7E00
:104FCE0020A3FD1F419DC3217FFCA2401E5F01E374
:104FDE00BD3E6082DC237D9FC1421CFEA0E1BF5D11
:104FEE000380DE3C62BEE0025CDF81633D7C22C05A
:104FFE009E1D43A1FF4618FAA427799BC584DA3873
:10500E0066E5BB5907DB856739BAE406581947A52B
:10501E00FB7826C49A653BD987045AB8E6A7F91BD4
:10502E0045C6987A24F8A6441A99C7257B3A648611
:10503E00D85B05E7B98CD2306EEDB3510F4E10F23E
:10504E00AC2F7193CD114FADF3702ECC92D38D6FDB
:10505E0031B2EC0E50AFF1134DCE90722C6D33D1A8
:10506E008F0C52B0EE326C8ED0530DEFB1F0AE4CC1
:10507E001291CF2D73CA947628ABF517490856B402
:10508E00EA6937D58B5709EBB536688AD495CB29A3
:10509E0077F4AA4816E9B7550B88D6346A2B75975C
:1050AE00C94A14F6A8742AC896154BA9F7B6E80A89
:1050BE0054D7896B35000000002B6096CBDDEE00D7
:0950CE002C96CBDDE5EEF7FAFDAE
:05691E00C1B101720A85
:1070DA0074FFF517F516F515F514AF17AE16AD15BD
:0270EA00AC14E4
:0170EC002281
:1060D90015701570A870ECF608EDF61570157015A9
:1060E90070A870C6EBC608C6EAC608C6E9C6E57058
:0460F90024FCF5701E
:1060FD00F80808E4F6A870F608F6E5702407F9A884
:10610D0070E6FE08E6FFC3099719E76480F8EE64B0
:10611D0080985037E5702404F8CBE6CB08E6FA08F2
:10612D00E6F98F828E83121207A870080866FFE5C4
:10613D00702403F8EFF6E6904FC393A8700808F6A5
:10614D00A8700806E61870B20680AFA8700808E6B9
:01615D00FF42
:07615E00E5702409F5702231
:0B716600ED6F78A7F6E6904FC393FF93
:0171710022FB
:0300A3000269846B
:10698400C0E0C083C082C0D0E8C0E0EEC0E0EFC089
:10699400E0E59830E1055398FDD231E59830E024E4
:1069A4007871E62401FFE433FEEF64404E70028008
:1069B400107871E6062445F582E43402F583E599FE
:1069C400F05398FED0E0FFD0E0FED0E0F8D0D0D075
:0669D40082D083D0E03206
:0A5E06008B438A4489458C468D4782
:105E1000E47871F6758401D284E54824FF929BE40E
:105E200078A8F678A8E6C39547E5466480F87480BC
:055E3000985060C23132
:0D5E3500754914754A1300D54AFCD549F68D
:105E4200E54724FFFFE54634FFFE78A8E66F7001C0
:105E5200EE701EC2ACAB430545E545AA447002058F
:105E62004414F91211EEF5993031FDC284D2AC809E
:105E720016AB430545E545AA447002054414F912E0
:105E820011EEF5993031FD7F01126E8778A80680F8
:055E920090C284AF473F
:015E970022E8
:0A5A90008B418A4289438C448D4506
:105A9A001270ED78A91214B3E478A8F61270EDEC3E
:105AAA00C0E0EDC0E0EEC0E0EFC0E078A912145209
:105ABA00CBEFCBCAEECAC9EDC9C8ECC8D0E0FFD05B
:105ACA00E0FED0E0FDD0E0FCC3EF9BFFEE9AFEEDD6
:105ADA0099FDEC98FCE47B01FAF9F8C31213C4505F
:105AEA00037F00227871E6FED3940040539002456A
:105AFA00E0FDB478037F0122ED54F8647860037FF7
:105B0A000022900245E05407240278A8F66E70300D
:105B1A007871E6D39545E5446480F8748098400628
:105B2A00AE44AF4580067871E6FF7E00A843AC42DA
:105B3A00AD417B017A0279451211C878A8E6FF22A5
:085B4A007F01126E87025AA6CA
:07000300E47871F6D231220E
:106AD300EF7025F5847598D0F584759115F5847557
:106AE300C90875CBFFED9050C293F5CA75C804E48D
:106AF300F584D2ACC2BC80267584017598D0E4F5C8
:106B030084E589540F4420F589758E02ED9050CCAD
:106B130093F58DD28E43E74043F740120003D2AF83
:016B2300224F
:1065D9009002851214CB000000009002891214CB9E
:1065E9000000000090023C7464F0E478A8F678A8F2
:1065F900E6FFC394025043EF25E025E0243DF582F0
:10660900E43402F583E4F0EF25E025E0243EF58249
:10661900E43402F583E4F0EF25E025E0243FF58238
:10662900E43402F583E4F0EF25E025E02440F58227
:0A663900E43402F583E4F00680B4B7
:016643002234
:106F9E00D2AFD2A9C2BBE4F584E589540F4401F502
:0F6FAE0089758E02758CAFE4F58AD28C0265D995
:025535001570EF
:10553700A870E4F6A870E6FFC3940240030256245D
:10554700EF25E025E02440F582E43402F583E0FF0F
:10555700D3940050030255F9E625E025E0243EF5F3
:1055670082E43402F583E060030255F9EF30E01975
:10557700E6FF25E025E02440F582E43402F583E0E8
:10558700D3940140047D0080067D01A870E6FF12D8
:1055970064FFA870E6FF25E025E02440F582E434A7
:1055A70002F583E0B401057D011264FFA870E6FFF0
:1055B70025E025E02440F582E43402F583E014F089
:1055C700EF25E025E02440F582E43402F583E0602E
:1055D70021E6FF25E025E0243FF582E43402F58348
:1055E700E0FEEF25E025E0243EF582E43402F58372
:1055F700EEF0A870E6FF25E025E0243EF582E434CE
:1056070002F583E06011EF25E025E0243EF582E412
:0D5617003402F583E014F0A8700602553B44
:03562400057022EC
:03000B00025D6B28
:105D6B00C0E0C0F0C083C082C0D0E8C0E0E9C0E0B2
:105D7B00EAC0E0EBC0E0ECC0E0EDC0E0EEC0E0EF6D
:105D8B00C0E0758CAF900285E0FCA3E0FDA3E0FEC4
:105D9B00A3E02401FFE43EFEE43DFDE43CFC900265
:105DAB00851214BF90023CE014F0E070259002893C
:105DBB00E0FCA3E0FDA3E0FEA3E02401FFE43EFE34
:105DCB00E43DFDE43CFC9002891214BF90023C744C
:105DDB0064F0125535126F7CD0E0FFD0E0FED0E0BE
:105DEB00FDD0E0FCD0E0FBD0E0FAD0E0F9D0E0F859
:0B5DFB00D0D0D082D083D0F0D0E032B6
:106E5A001570A870EDF61570A870EFF6A870E6FF29
:106E6A00C39402501308E6FEEF25E025E0243DF521
:0D6E7A0082E43402F583EEF005700570220D
:105E980015701570A870EAF608EBF61570A870ED85
:105EA800F61570A870EFF6A870E6FFC39402506A62
:105EB800EF25E025E02440F582E43402F583E07024
:105EC80059E6FB25E025E0243EF582E43402F5831B
:105ED800E0704708E625E004FFA870E6FA25E0250B
:105EE800E02440F582E43402F583EFF00808E6FE8A
:105EF80008E6FF7C007D0A1212CFEA25E025E0249F
:105F08003FF582E43402F583EFF0EB25E025E02449
:105F18003EF582E43402F583E4F0E5702404F5707C
:015F28002256
:0E64FF001570A870EDF61570A870EFF6157008
:10650D00A87008E6FFC394025024EF25E025E0248F
:10651D003DF582E43402F583E06013A8700808E6C7
:10652D0070047F0180027F00A8700808EFF6A87044
:10653D00A68475840FA87008E6FF700BA870080874
:10654D00E624FF9286800DEFB40109A8700808E6D5
:09655D0024FF9287A870E6F58482
:0765660005700570057022AD
:1070ED00C2AF900285E0FCA3E0FDA3E0FEA3E0FFAC
:0270FD00D2AF10
:0170FF00226E
:10710000C2AF900289E0FCA3E0FDA3E0FEA3E0FF94
:02711000D2AFFC
:01711200225A
:106E87001570A870EFF6A870E670057873F608F627
:106E97003030167872E675F064A4FFC37874E69F05
:0C6EA70018E695F0500375FFA505702259
:106FBD00D230E47873F608F6EF78726003F680024B
:0F6FCD00760A75FF0775FFA5E4F58475EF0422BA
:10711300C230E47873F608F6787276FF75FFDE7591
:03712300FFAD229B
:106F7C00787406E6187001063030167872E675F0F3
:106F8C0064A4FFC37874E69F18E695F0500375FF70
:026F9C00A5222C
:046EB3008E448F4535
:106EB700E4F546F547C3E5479545E546954450163D
:106EC7007FE87E031267787F01126E870547E547E3
:066ED70070E3054680DFB8
:016EDD002292
:046778008E658F6635
:10677C00D3E56694FAE56594005010AF66EFD394B8
:10678C000040407E1600DEFD1F80F2856567856641
:10679C0068D3E56894FAE567940040157FFA7E00AB
:1067AC0012677874062568F56874FF3567F567809D
:1067BC00E0D3E5669400E56594004007AF68AE67EA
:0367CC00126778D9
:0167CF0022A7
:1066AF0075500075510075524A7B007A0079487D0C
:0166BF0002D8
:0866C0008B4C8A4D894E8D4F71
:1066C8007F01126E87AB50AA51A9521213052400FC
:1066D800FFE5F034E0FE854C53854D54854E55E476
:1066E800FDEDC3954F501BEF2DF582E43EF583E495
:1066F80093AB53AA54A9558D827583001212460D87
:0F67080080DFAB50AA51A952E4854FF00213680D
:105C1300754112754234754900754A00754B437BD3
:075C2300007A0079417D02C7
:085C2A008B458A4689478D482D
:105C32007880E664F16003025CC7127113C2AFE4BC
:105C4200F58443B701758F01AB49AA4AA94B1213D8
:105C5200052400FFE5F034E078A8F608EFF6AA463E
:105C6200A94778ACA64508C6EAC608C6E9C6E478DC
:105C7200AAF678AAE6C39548503278ACCBE6CB08B0
:105C82000806E618CAE6CA70010614F91211EE787F
:105C9200ABF6E6FF78A80806E618CCE6CC7001065B
:105CA20014F5828C83EFF078AA0680C6E4F58F5350
:105CB200B7F0AB49AA4AA94B8548F0121368D2AF94
:055CC200E4FF126FBDBC
:015CC70022BA
:106B74007880E664F17046C2AF127113E4F5844381
:106B8400B701758F0378A976E008F678A8F678A996
:106B9400E6FE08E6F5828E83E4F07F01126E8778C4
:106BA400AAE426F618740236F61806E6C3940840DA
:0D6BB400DDE4F58F53B7F0D2AFFF126FBDD7
:016BC10022B1
:105CC800126B74E4F543F544F549754A00754B4386
:105CD800FB7A00798D7D16125C2A125C13E4F5407C
:105CE800E540C37877965073E4F53FAB18AA19A935
:105CF8001A75F020E53FA4F58285F083121207603B
:105D080056E53F75F020A429F9EA35F0FA90000D20
:105D180012150C788AE68540F0A429F9EA35F0FADC
:105D2800EBC0E0EAC0E0E9C0E0AB18AA19A91A750F
:105D3800F020E53FA4F58285F083121207FD75492E
:105D480000754A00754B43D0E0F9D0E0FAD0E0FB8B
:105D5800125C2A053F809405408085125C13E47824
:025D680080F6C3
:015D6A002216
:025627008F44AE
:10562900E4F54AF54BF547F55075510075524AFBBB
:105639007A00798D7D161266C01266AFE549643429
:105649007004E54864127003434701E4F546E546F2
:10565900C378779640030256FAE4F545AB18AA19C0
:10566900A91A75F020E545A4F58285F08312120781
:10567900607AE5446054E54575F020A429F9EA35D6
:10568900F0FA90000D12150C788AE68546F0A429E7
:10569900F9EA35F0FAEBC0E0EAC0E0E9C0E0AB189E
:1056A900AA19A91A75F020E545A4F58285F0831297
:1056B9001207FD75500075510075524AD0E0F9D0B6
:1056C900E0FAD0E0FB1266C0801DAB18AA19A91A2E
:1056D90075F020E545A4F58285F083121207254B64
:1056E900F54BE4354AF54A05450256650546025625
:1056F900571266AFE54964347004E54864127003D3
:05570900434702AF4719
:01570E002278
:106FFA00EF540778AAF6EF30E306E64420F6800459
:0C700A0078AAE6F678AAE644C0F6F5C8BD
:017016002257
:02477B008F4469
:10477D001271597D017F021270C67BFF7A4F799EAF
:10478D00122FB6E478A9F6127113C2AFE478A8F629
:10479D0078A8E6FFC3954440030248DE126FFA780D
:1047AD00A8E6FF7D031270C67FDA1270B09020006C
:1047BD00AF82AE83C3EF94FFEE94FF5005E4F0A3F8
:1047CD0080EE902000AF82AE83C3EF94FFEE94FF96
:1047DD00500CE0600678A976018003A380E778A9E4
:1047ED00E660030248DE78A8E6FF7D031270C67FFF
:1047FD00D91270B0902000AF82AE83C3EF94FFEE5C
:10480D0094FF50067455F0A380ED902000AF82AE5A
:10481D0083C3EF94FFEE94FF500EE064556006786D
:10482D00A976018003A380E578A9E660030248DE3E
:10483D0078A8E6FF7D031270C67FD81270B0902065
:10484D0000AF82AE83C3EF94FFEE94FF500674AABF
:10485D00F0A380ED902000AF82AE83C3EF94FFEE06
:10486D0094FF500EE064AA600678A976018003A338
:10487D0080E578A9E6705A78A8E6FF7D031270C628
:10488D007FD71270B0902000AF82AE83C3EF94FF3C
:10489D00EE94FF500674FFF0A380ED902000AF82E0
:1048AD00AE83C3EF94FFEE94FF500DE0F4600678F5
:1048BD00A976018003A380E678A9E6701478A8E6AE
:1048CD00FF7D031270C67FD61270B078A80602471E
:1048DD009DD2AFE4FF126FBD126FFA78A9E6601B8F
:1048ED007D02E41270C67BFF7A4F79AD78A8E6F5AC
:0B48FD0049122FB67F00126E8780F971
:01490800228C
:10664400E4F58475A338F5A275A10475840F759CCF
:10665400FF759DFF759EFF759FFF75F8FF75E8FF39
:1066640075D8FF75C8FFFF126FFA902000E078A874
:10667400F67455F0E064556008E6F0E4F584F5A39B
:106684002278A8E6F07F08126FFAE078A8F674AAD8
:10669400F0E0B4AA0AE6F0E4FF126FFA7F10227861
:0A66A400A8E6F0E4FF126FFA7F0889
:0166AE0022C9
:1033C300202020202020202020200025622A626443
:1033D3000025622A62750025622A640025622A7527
:1033E3000025622A2E622A660025622A6C64002563
:1033F300622A6C7500253262753A257300202020FD
:103403002020202020004E6F207661726961626C5B
:10341300657320646566696E656400202020202042
:103423002020202020202020202020202020004594
:10343300534320454E5445522020202D2020202048
:103443002B20200045534320454E54455220202035
:103453002D20202020202B200045534320454E546F
:1034630045522020200045534320202020202020A7
:103473002020002020202020002000506172616D58
:103483006574657273207772697474656E00746F06
:1034930020666C617368206D656D6F72792E00F420
:1034A30070000000F76E000000FA8F000000FD6D51
:1034B3000000000000000000036B000000064D0048
:1034C300000009470000000C5400000063000000E6
:1034D30000016D000000026700000003730000009C
:1034E300046D0000000568000000064100000007AD
:1034F3004B00000008804300000980460000144888
:103503007A00001550610000166261000017570031
:103513000000185600000019B50000001A540000FE
:10352300001B6C2F73001C52504D001D4600000001
:103533001E4A0000005A250000005B52504D005CFB
:10354300636E74005D780000000000000000023527
:103553000000004E6F64652041647200008D01001D
:10356300000000000000003F800000000000023562
:10357300000000477270204164720000008F010058
:10358300000000000000003F8000000000000A3837
:1035930000000054696D65000000000102D30100C2
:1035A300000000000000003F8000000000000A3817
:1035B30000000044617465000000000102C30100C3
:1035C300000000000000003F80000000000004082D
:1035D30000000154656D700000000001029B0200B1
:1035E300000000000000003F8000000000000418FD
:1035F300000001312E3856000000000102B3020022
:10360300000000000000004000000000000004185B
:10361300000001332E33560000000001029F020018
:10362300000000000000004000000000000004183B
:1036330000000135566578740000000102A70200FE
:10364300000000000000004000000000000004181B
:1036530000000132345600000000000102AB0200FA
:10366300000000000000003F80000000000004187C
:1036730000000132345665787400000102AF020085
:10368300000000000000003F80000000000004066E
:1036930000000149203234560000000102A3020059
:1036A30000000000000000400000000000000032A5
:1036B300000004466C617368000000000000000015
:1036C30000000000000000000000000000000032C5
:1036D3000000045265626F6F740000000000000078
:0E36E3000000000000000000000000000000D9
:0A692300C19FC127C126C120C12178
:0639BE008B408A418942A2
:1039C4009000011212076438705985434985444AAE
:1039D40085454BF54C754D0A7B017A0279B7126A1D
:1039E400307B017A0279B712000EC3EF940AEE9489
:1039F40000502DE49002EBF07B017A0279B71200BB
:103A04000EC3740A9FFFE49EFE9002EBE0C39FE4A2
:103A14009E500D7F201270B09002EBE004F080D82D
:103A2400023C7EE49002B7F0AB40AA41A942900068
:103A3400021212076068E49002EBF09002EBE0756A
:103A4400F005A424A2F582E43434F583E493FF64FE
:103A5400636019AB40AA41A942900002121207FE0A
:103A6400EF6E60089002EBE004F080CF9002EBE090
:103A7400FF75F005A424A2F582E43434F583E493BD
:103A8400601CEF75F005A424A3F9743435F075496E
:103A9400FFF54A894B7B017A0279B7126828AB405B
:103AA400AA41A9429000011212076066E49002EB59
:103AB400F09002EBE075F005A424D4F582E43434EC
:103AC400F583E493FF6019AB40AA41A94290000139
:103AD400121207FEEF6E60089002EBE004F080D152
:103AE4009002EBE0FF75F005A424D4F582E43434AD
:103AF400F583E493601CEF75F005A424D5F97434C0
:103B040035F07549FFF54A894B7B017A0279B71282
:103B140068287B017A0279B712000E9002ECEFF06C
:103B2400AB40AA41A9421211EE14601D1460642432
:103B3400FE7003023BE724046003023C7E7BFF7AB1
:103B44003379C3126EDE023C7EAB40AA41A9429097
:103B540000041212079002EC30E11CE0FFC3740A67
:103B64009FF549AB43AA44A9451211EEF54A7BFFE0
:103B74007A3379CE023C7BE0FFC3740A9FF549ABEC
:103B840043AA44A9451211EEF54A7BFF7A3379D44E
:103B9400023C7BAB40AA41A9429000041212079058
:103BA40002EC30E11FE0FFC3740A9FF549AB43AA5E
:103BB40044A945121305F54B85F04A7BFF7A337906
:103BC400DA023C7BE0FFC3740A9FF549AB43AA4485
:103BD400A945121305F54B85F04A7BFF7A3379DF4B
:103BE400023C7BAB40AA41A9429000041212073068
:103BF400E0339002ECE0FFC3740A9FF54990001093
:103C0400121207FF600280027F038F4AAB43AA446B
:103C1400A9451213E88F4E8E4D8D4C8C4B7BFF7A49
:103C24003379E48052AB40AA41A9429000041212B5
:103C3400079002EC30E121E0FFC3740A9FF549AB21
:103C440043AA44A9451213E88F4D8E4C8D4B8C4AE0
:103C54007BFF7A3379EC801FE0FFC3740A9FF54938
:103C6400AB43AA44A9451213E88F4D8E4C8D4B8C5F
:103C74004A7BFF7A3379F2122FB67B017A0279B745
:033C8400126EDEDF
:013C8700221A
:0D1F33009002DEE0FBA3E0FAA3E0F97DFFE1
:101F40008D438B408A418942900001121207643808
:101F50007003022744AB40AA41A9421211EE24FEAD
:101F600070030221A524FE70030223FE24036003F4
:101F700002274490000412120720E10302205FAB05
:101F800040AA41A942900019121483C000C001C0A8
:101F900002C003AC43EC120EA1D003D002D001D09A
:101FA00000120C78C004C005C006C00790028DE086
:101FB000FC120EA1D003D002D001D000120B871268
:101FC0000ED590028DEFF0AB40AA41A942900015CA
:101FD000121408900011121483120E1E70030227AF
:101FE00044AB40AA41A942900011121408C004C099
:101FF00005C006C00790028DE0FC120EA1A804A93E
:1020000005AA06AB07D007D006D005D004120E1ED5
:102010005014AB40AA41A942900011121408120EAC
:10202000D590028DEFF0AB40AA41A9429000151265
:102030001408C004C005C006C00790028DE0FC1261
:102040000EA1A804A905AA06AB07D007D006D005A3
:10205000D004120E1E60025003022744022190E5B4
:1020600043F4704CAB40AA41A942900011121408ED
:10207000C004C005C006C00790028DE0FCE4120E4B
:10208000A1A804A905AA06AB07D007D006D005D0A1
:1020900004120E1E701AAB40AA41A94290001512FC
:1020A0001408900011121483120E1E6003022744BC
:1020B000AB40AA41A942900019121483C000C0018C
:1020C000C002C003AC43EC120EA1D003D002D00179
:1020D000D000120C78C004C005C006C00790028D65
:1020E000E0FCE4120EA1D003D002D001D000120B0C
:1020F00087120ED590028DEFF0AB40AA41A9429015
:102100000015121408900011121483120E1E700391
:10211000022744AB40AA41A942900011121408C002
:1021200004C005C006C00790028DE0FCE4120EA1B9
:10213000A804A905AA06AB07D007D006D005D0048D
:10214000120E1E5014AB40AA41A942900011121465
:1021500008120ED590028DEFF0AB40AA41A9429033
:102160000015121408C004C005C006C00790028DF7
:10217000E0FCE4120EA1A804A905AA06AB07D0074B
:10218000D006D005D004120E1E6002500302274470
:10219000AB40AA41A942900015121408120ED59026
:1021A000028DEFF022AB40AA41A942900004121226
:1021B0000720E1030222A3900019121483C000C07B
:1021C00001C002C003AC43EC120EA1D003D002D078
:1021D00001D000120C78C004C005C006C0079002F0
:1021E0008DE0FCA3E0FDEC120E9CD003D002D001E8
:1021F000D000120B87120ED590028DEEF0A3EFF0F7
:10220000AB40AA41A9429000151214089000111287
:102210001483120E1E7003022744AB40AA41A94248
:10222000900011121408C004C005C006C007900237
:102230008DE0FCA3E0FDEC120E9CA804A905AA0603
:10224000AB07D007D006D005D004120E1E5017AB36
:1022500040AA41A942900011121408120ED5900212
:102260008DEEF0A3EFF0AB40AA41A9429000151209
:102270001408C004C005C006C00790028DE0FCA38E
:10228000E0FDEC120E9CA804A905AA06AB07D00736
:10229000D006D005D004120E1E600250030227445F
:1022A0000223E6E543F4704FAB40AA41A9429000F7
:1022B00011121408C004C005C006C00790028DE0CA
:1022C000FCA3E0FDE4120E9CA804A905AA06AB0736
:1022D000D007D006D005D004120E1E701AAB40AA4B
:1022E00041A9429000151214089000111214831293
:1022F0000E1E6003022744AB40AA41A94290001978
:10230000121483C000C001C002C003AC43EC120E23
:10231000A1D003D002D001D000120C78C004C005B7
:10232000C006C00790028DE0FCA3E0FDE4120E9C05
:10233000D003D002D001D000120B87120ED590022C
:102340008DEEF0A3EFF0AB40AA41A9429000151228
:102350001408900011121483120E1E7003022744F9
:10236000AB40AA41A942900011121408C004C00554
:10237000C006C00790028DE0FCA3E0FDE4120E9CB5
:10238000A804A905AA06AB07D007D006D005D0043B
:10239000120E1E5017AB40AA41A942900011121410
:1023A00008120ED590028DEEF0A3EFF0AB40AA41DB
:1023B000A942900015121408C004C005C006C00749
:1023C00090028DE0FCA3E0FDE4120E9CA804A90598
:1023D000AA06AB07D007D006D005D004120E1E60A7
:1023E000025003022744AB40AA41A94290001512B3
:1023F0001408120ED590028DEEF0A3EFF022AB4040
:10240000AA41A94290000412120720E0030224C04E
:1024100090028DE0F8A3E0F9A3E0FAA3E0FBC0008E
:10242000C001C002C003AB40AA41A94290001912EA
:102430001483C000C001C002C003AC43EC120EA163
:10244000D003D002D001D000120C78D003D002D03B
:1024500001D000120B8790028D1214BFAB40AA412D
:10246000A94290001112140890028DE0F8A3E0F93F
:10247000A3E0FAA3E0FB120E1E5012AB40AA41A942
:102480004290001112140890028D1214BFAB40AAA2
:1024900041A94290001512140890028DE0F8A3E0C3
:1024A000F9A3E0FAA3E0FB120E1E6002500302271C
:1024B00044AB40AA41A94290001512140802273EDD
:1024C000AB40AA41A94290000412120720E1030286
:1024D00025DB900019121483C000C001C002C003A4
:1024E000AC43EC120EA1D003D002D001D000120CEC
:1024F00078C004C005C006C00790028DE0FCA3E0D0
:10250000FDA3E0FEA3E0FFEC120E97D003D002D0B3
:1025100001D000120B87120ED590028D1214BFABA2
:1025200040AA41A9429000151214089000111214FB
:1025300083120E1E7003022744AB40AA41A94290A9
:102540000011121408C004C005C006C00790028D17
:10255000E0FCA3E0FDA3E0FEA3E0FFEC120E97A8D1
:1025600004A905AA06AB07D007D006D005D00412EF
:102570000E1E5015AB40AA41A9429000111214083A
:10258000120ED590028D1214BFAB40AA41A9429001
:102590000015121408C004C005C006C00790028DC3
:1025A000E0FCA3E0FDA3E0FEA3E0FFEC120E97A881
:1025B00004A905AA06AB07D007D006D005D004129F
:1025C0000E1E60025003022744AB40AA41A942906C
:1025D0000015121408120ED502273EE543F470557B
:1025E000AB40AA41A942900011121408C004C005D2
:1025F000C006C00790028DE0FCA3E0FDA3E0FEA3AF
:10260000E0FFE4120E97A804A905AA06AB07D007BD
:10261000D006D005D004120E1E701AAB40AA41A9F4
:1026200042900015121408900011121483120E1E0D
:102630006003022744AB40AA41A94290001912143A
:1026400083C000C001C002C003AC43EC120EA1D095
:1026500003D002D001D000120C78C004C005C0061F
:10266000C00790028DE0FCA3E0FDA3E0FEA3E0FF25
:10267000E4120E97D003D002D001D000120B8712C3
:102680000ED590028D1214BFAB40AA41A942900012
:1026900015121408900011121483120E1E700302FA
:1026A0002744AB40AA41A942900011121408C0046B
:1026B000C005C006C00790028DE0FCA3E0FDA3E0CA
:1026C000FEA3E0FFE4120E97A804A905AA06AB0733
:1026D000D007D006D005D004120E1E5015AB40AA6C
:1026E00041A942900011121408120ED590028D12C9
:1026F00014BFAB40AA41A942900015121408C004AF
:10270000C005C006C00790028DE0FCA3E0FDA3E079
:10271000FEA3E0FFE4120E97A804A905AA06AB07E2
:10272000D007D006D005D004120E1E60174015AB9E
:1027300040AA41A942900015121408120ED5900229
:052740008D1214BF2200
:106CA1008F40E92405F9E43AFA78B77C027D017E48
:106CB100007F081211C8E49002BFF09002BDE0FF0E
:106CC10060079002BCF0E4A3F0854049754A017564
:106CD1004B02754CB77BFF7A3379F8122FB67BFFE5
:076CE1007A347900026EDE37
:1000A600123C88EF6003D21F22301F40E490029A70
:1000B600F09002921214CB000000009002961214E7
:1000C600CB00000000C222C223C224C225E4900253
:1000D600E4F01270EDE47B2C7A01F9F8C31213C434
:1000E6004003020B7FC21FD21412418120271EC279
:1000F600141241819002E4EFF07003020B6FD227D5
:10010600E064026003020B6FD226020B6F20260307
:100116000204DD9002C3742DF0E4A3F09002D374C0
:100126002DF0E4A3F07544017545027546E5754763
:1001360002FB7D02FF124E639002E5E0C4F854F024
:10014600C868FCA3E0C4540F48FDE4120E9CE4FB0F
:10015600FAF97841120D819002E71214BFE4FFFE0E
:100166007D207C419002E7E0F8A3E0F9A3E0FAA342
:10017600E0FB120C78E4FBFAF9783F120B87120EBB
:10018600D5EC120E97E4FBFA79207841120D819096
:10019600029B1214BF7544017545027546E5754705
:1001A600027B017D02E4FF124E639002E5E0C4F893
:1001B60054F0C868FCA3E0C4540F48FDE4120E9C3A
:1001C600E4FBFA79A07840120C78E4FBFA7980789F
:1001D60045120D819002E71214BFE4FFFE7DC87C34
:1001E600429002E7E0F8A3E0F9A3E0FAA3E0FB12ED
:1001F6000C78E4FBFAF9783F120B87120ED5EC1255
:100206000E97E4FBFA79C87842120D8190029F128C
:1002160014BF7544017545027546E57547027B02B4
:100226007D02E4FF124E639002E5E0C4F854F0C884
:1002360068FCA3E0C4540F48FDE4120E9CE4FBFAEC
:1002460079207840120C78E4FBFA79807845120D13
:10025600819002E71214BF9002E7E0FCA3E0FDA341
:10026600E0FEA3E0FF7B007AC079287845120D8175
:100276009002E71214BF9002E7E0FCA3E0FDA3E0C2
:10028600FEA3E0FF7B007AC0795A7846120C78907C
:1002960002E71214BFE4FFFE7DC87C429002E7E04D
:1002A600F8A3E0F9A3E0FAA3E0FB120C78E4FBFA6A
:1002B600F9783F120B87120ED5EC120E97E4FBFA73
:1002C60079C87842120D819002A31214BF754401B9
:1002D6007545027546E57547027B037D02E4FF120C
:1002E6004E639002E5E0C4F854F0C868FCA3E0C48D
:1002F600540F48FDE4120E9CE4FBFA79C8784012CC
:100306000C78E4FBFA79807845120D819002E712A9
:1003160014BFE4FFFE7DC87C429002E7E0F8A3E04C
:10032600F9A3E0FAA3E0FB120C78E4FBFAF9783FB4
:10033600120B87120ED5EC120E97E4FBFA79C878E9
:1003460042120D819002A71214BF75440175450231
:100356007546E57547027B047D02E4FF124E639005
:1003660002E5E0C4F854F0C868FEA3E0C4540F48A0
:10037600FF7C007D0B121268AC06AD07E4120E9CE2
:10038600E4FBFA79207840120C78E4FBFA7980785D
:1003960045120D819002E71214BFE4FFFE7DC87C72
:1003A600429002E7E0F8A3E0F9A3E0FAA3E0FB122B
:1003B6000C78E4FBFAF9783F120B87120ED5EC1293
:1003C6000E97E4FBFA79C87842120D819002AB12BF
:1003D60014BF7544017545027546E57547027B05F0
:1003E6007D02E4FF124E639002E5E0C4F854F0C8C3
:1003F60068FEA3E0C4540F48FF7C007D0B12126810
:10040600AC06AD07E4120E9CE4FBFA7920784012A4
:100416000C78E4FBFA79807845120D819002E71298
:1004260014BFE4FFFE7DC87C429002E7E0F8A3E03B
:10043600F9A3E0FAA3E0FB120C78E4FBFAF9783FA3
:10044600120B87120ED5EC120E97E4FBFA79C878D8
:1004560042120D819002AF1214BF75440175450218
:100466007546E57547027B067D02E4FF124E6390F2
:1004760002E5E0C4F854F0C868FCA3E0C4540F4891
:10048600FDE4120E9CE4FBFA79207840120C78E425
:10049600FBFA79807845120D819002E71214BFE4C9
:1004A600FFFE7DC87C429002E7E0F8A3E0F9A3E0F6
:1004B600FAA3E0FB120C78E4FBFAF9783F120B87FB
:1004C600120ED5EC120E97E4FBFA79C87842120D9B
:1004D600819002B31214BF9002DE30261374FFF02F
:1004E600A37435F0A37451F09002E2740CF08013FB
:1004F600E518F0A3E519F0A3E51AF07882E6149062
:1005060002E2F09002E2E0FFC394035005E4A3F098
:10051600801B90029AE0FE7002800EEE90029AB561
:100526000705E024FE8002E0149002E3F07882E6FC
:100536007014202611FDFF1270C67BFF7A347909EC
:10054600122FB6020695E49002E1F09002E1E0FD7A
:10055600C394034003020695E4FF1270C69002E1BD
:10056600E0FF9002E3E02FFFE433FE90029AE07C86
:1005760000B50708ECB506047F1580027F201270CF
:10058600B09002E1E0FD7F011270C69002E1E0FF4B
:100596009002E3E02FFFE433FE9002E2E0FDD3EFAA
:1005A6009D7480F86E98400C7BFF7A34791E122F6A
:1005B600B602068C9002E1E0FE9002E3E0FD2EFF1B
:1005C600C007EEFFED2FFFE433FEEF7805C333CE11
:1005D60033CED8F9FF9002DEE0FBA3E0FAA3E02FCA
:1005E600F9EA3EFAD007126CA19002E1E0FD7F0A1B
:1005F6001270C63020409002E1E0FF9002E3E02F47
:10060600FFE433FE90029AE07C00B50729ECB506BC
:1006160025EF7805C333CE33CED8F9FF9002DEE05E
:10062600FBA3E0FAA3E02FF9EA3EFA75430175440D
:100636000275458D804D9002E1E0FF9002E3E02FC8
:10064600FFE433FEEF7805C333CE33CED8F9FF90FF
:1006560002DEE0FBA3E0FAA3E02FF9EA3EFAC003CC
:10066600C002C0019002DEA3E0FAA3E02FF9EA3E41
:10067600FA90000D12150C8B438A448945D001D09F
:1006860002D0031239BE9002E1E004F00205519057
:10069600029AE075F020A430260F2451F9743535FE
:1006A600F0FA9002DE74FF800D251AF9E51935F08F
:1006B600FA9002DEE518F0A3EAF0A3E9F030215A39
:1006C6007D03E4FF1270C67BFF7A347932126EDE48
:1006D600900291E075F003A4240DFF9002E3E0FE82
:1006E60090029AE0C39EFD1270C620080A302207C7
:1006F600C221E4FF127139200903020B6F30230374
:10070600020B6F900291E004F0E064036003020BB9
:100716006FC221FF127139020B6F2020030208E419
:100726007D03E4FF1270C67BFF7A347947126EDED2
:100736009002E3E0FF90029AE0C39FFD7F131270E0
:10074600C620080A302207C220E4FF127139300998
:1007560053202350C220E4FF1271399002DEE0FBE1
:10076600A3E0FAA3E0F91211EEFF7E009002DEA3E9
:10077600A3E090000D12150CA801AC02AD037B019D
:100786007A02798D1211C830261290029AE0FF6023
:1007960003B40110D228788076F1800890029AE09E
:1007A600FF126F57300A0F20240C121F331270ED00
:1007B6009002921214BF300A2D1270EDA804A905FA
:1007C600AA06AB07900292E0FCA3E0FDA3E0FEA31D
:1007D600E02446FFE43EFEE43DFDE43CFCD3121378
:1007E600C44003121F33300A3B1270EDA804A9055A
:1007F600AA06AB07900292E0FCA3E0FDA3E0FEA3ED
:10080600E024F4FFEE3401FEE43DFDE43CFCD312AB
:1008160013C440109002DEE0FBA3E0FAA3E0F97DEA
:10082600F7121F40200A0A9002921214CB00000011
:1008360000300B1C2025199002DEE0FBA3E0FAA392
:10084600E0F97D01121F401270ED9002961214BF5E
:10085600300B3A1270EDA804A905AA06AB07900260
:1008660096E0FCA3E0FDA3E0FEA3E02446FFE43E01
:10087600FEE43DFDE43CFCD31213C440109002DEBE
:10088600E0FBA3E0FAA3E0F97D01121F40300B3B29
:100896001270EDA804A905AA06AB07900296E0FC23
:1008A600A3E0FDA3E0FEA3E024F4FFEE3401FEE4A2
:1008B6003DFDE43CFCD31213C440109002DEE0FB85
:1008C600A3E0FAA3E0F97D09121F40300B03020BE7
:1008D6006F9002961214CB00000000020B6F7D038E
:1008E600E4FF1270C67882E6D394005003302637B0
:1008F6009002DEE0FBA3E0FAA3E0F99000191214DF
:1009060008E4FBFAF9F8120E1E40149002DEE0FB32
:10091600A3E0FAA3E0F990000412120730E2087B84
:10092600FF7A34795C80067BFF7A347969126EDE51
:100936007F121270B07BFF7A347976126EDE7F13E7
:100946001270B07BFF7A34797C126EDE20080C3090
:100956002209C227C226D214124181200903020AA3
:100966004D302303020A4D7882E6D394004061900D
:1009760002DEE0FBA3E0FAA3E0F91211EEFFD39446
:1009860004504DEF94004048900019121408E4FBFF
:10099600FAF9F8120E1E5038D2209002DEE0FBA3C0
:1009A600E0FAA3E0F91211EEFF7E0090000D121599
:1009B6000C788D7C027D011211C89002E3E0FF9055
:1009C600029AE0C39FFD7F131270C67F0112713930
:1009D60030262A90029AE0FF64026004EFB4031DF9
:1009E600D221E4900291F09002E3E0FF90029AE0B7
:1009F600C39FFD7F0D1270C67F01127139302637F5
:100A060090029AE0640B702FD228788076F11271EA
:100A160059E4FDFF1270C67BFF7A34797E126EDED2
:100A26007D01E4FF1270C67BFF7A347991126EDE87
:100A36007FB87E0B126EB330260D90029AE0B40C8E
:100A460006E4F58475EF10300A2A20242790029ACE
:100A5600E070122026077882E614F0800E90029A43
:100A6600740CF0800690029AE014F01270ED900279
:100A7600921214BF300A481270EDA804A905AA06FE
:100A8600AB07900292E0FCA3E0FDA3E0FEA3E02406
:100A960046FFE43EFEE43DFDE43CFCD31213C440B5
:100AA6001E90029AE070122026077882E614F080E3
:100AB6000E90029A740CF0800690029AE014F020D0
:100AC6000A0A9002921214CB000000003026089009
:100AD60002E1740DF080077882E69002E1F0300BB7
:100AE6002520252290029AE02401FFE433FE90029D
:100AF600E1E0FD7C0012127A90029AEDF01270EDA0
:100B06009002961214BF300B431270EDA804A9058B
:100B1600AA06AB07900296E0FCA3E0FDA3E0FEA3C5
:100B2600E02446FFE43EFEE43DFDE43CFCD3121324
:100B3600C4401990029AE02401FFE433FE9002E1DA
:100B4600E0FD7C0012127A90029AEDF0200B0A90DA
:100B560002961214CB00000000300A0D300B0A205A
:100B66002607E490029AF0D226A2089222A20992BF
:090B760023A20A9224A20B92258D
:010B7F002253
:0267D0008F63D5
:1067D20075840FE4F5A6C290C294D295D2967F0139
:1067E200FE126778C296E4F5647F0A7E001267782B
:1067F20030A7090564E564C394C840ED75840F753C
:10680200A6FFD290C295A21E92948563A07F017EBC
:1068120000126778D2967F017E00126778C2967F57
:06682200017E0002677810
:10656D00D23275840F43A580C2977F017E00126ED3
:10657D00B3D2977F327E00126EB3C296C295C2948B
:10658D0075840F75A6FF43A503D290D291C21E7FCD
:10659D00341267D0C21E7F0B1267D0C21E7F30121D
:1065AD0067D0C21E7F021267D0C21E7F0C1267D049
:1065BD00C21E7F011267D0C21E7F341267D0C21E69
:0C65CD007F061267D0C21E7F300267D02C
:0D715900C21E7F011267D0E4FDFF0270C668
:10713900EF6006C21E7F0F8004C21E7F0C1267D04B
:017149002223
:1070C600ED5403C43354E0FEEF541F44804EFFC218
:0470D6001E0267D05F
:1070B0008F62E562640D600BE562640A6005D21EB2
:0670C0001267D0AF62224E
:106F30008B698A6A896BAB69AA6AA96B1211EE60C8
:106F400015056BE56B7002056A14F91211EEFFD29C
:076F50001E1267D080E02251
:044E63008D428B43AE
:104E67007B08E4FD127179E49002F3F0E5425408FF
:104E7700D394004003D38001C392B3000000000025
:104E8700000000000000000000000000000000D249
:104E9700B00000000000000000000000000000005B
:104EA7000000000000C2B0E54225E0F5429002F3A1
:104EB700E004F0E0B404B5E49002F3F0E5435408ED
:104EC700D394004003D38001C392B30000000000D5
:104ED700000000000000000000000000000000D2F9
:104EE700B00000000000000000000000000000000B
:104EF7000000000000C2B0E54325E0F5439002F34F
:104F0700E004F0E0B404B5E49002F3F0E54775F08F
:104F170008A4FF9002F3E0FDC39FE5F06480F874F6
:104F27008098505CED9400400FE05407700A042508
:104F370046F546E43545F545C2B0000000000000DF
:104F47000000000000000000000000000000AB446B
:104F5700AA45A9461211EE25E0FFA2B4E4334F1289
:104F67001234D2B000000000000000000000000072
:104F770000000000000000009002F3E004F0808CC5
:104F8700D2B2000000000000000000000000000096
:064F970000000000000014
:014F9D0022F1
:0458D9007D0AAF464F
:0458DD008D478B4820
:1058E100D2B2000000000000000000000000000033
:1058F100000000000000C2B2000000000000000033
:105901000000000000000000000000007B08E4FD32
:10591100127179E49002F3F0E5475408D394004002
:1059210003D38001C392B300000000000000000017
:105931000000000000000000000000D2B0000000E4
:105941000000000000000000000000000000000056
:1059510000C2B0E54725E0F5479002F3E004F0E02E
:10596100B404B5E49002F3F0E5485408D394004040
:1059710003D38001C392B3000000000000000000C7
:105981000000000000000000000000D2B000000094
:105991000000000000000000000000000000000006
:1059A10000C2B0E54825E0F5489002F3E004F0E0DC
:0359B100B404B586
:0159B40022D0
:106BC200E49002E6F0EF5480D394004003D38001B6
:106BD200C392B300000000000000000000000000AB
:106BE20000000000000000D2B00000000000000021
:106BF20000000000000000000000000000C2B0EF32
:0D6C020025E0FF9002E6E004F0E0B408B8E1
:016C0F002262
:025B52008F467C
:105B5400E4FB7D071258DDE4FB1258D9E4FF126B15
:105B6400C2E4FF126BC27B021258D9E4FF126BC26B
:105B7400E4FF126BC2E49002E3F09002E3E0FBC3A3
:105B8400940750697D0CAF461258DD9002E3E0FFA4
:105B9400700AA37403F0A37420F08017EF9002E45A
:105BA400B402097401F0A374D9F08007740FF0A350
:105BB40074FFF09002E4E0C4F854F0C8A3E0C454C5
:105BC4000F48FF126BC29002E5E0540FC4F8540F63
:105BD400C868FF126BC2E4FF126BC2E4FF126BC20F
:105BE4007F3A126BC29002E3E004F0808DE4FB7D07
:105BF4000DAF461258DD7FFF126BC27FFF126BC2DE
:0F5C0400E4FF126BC2E4FF126BC27F14026BC28B
:106FDC00E4FB7D091258DDD2B20000000000000075
:0E6FEC00000000000000000000000000002275
:046F08008F6C8D6D90
:106F0C007B017A037914126049E56D9003146006D5
:106F1C00E04401F08004E054FEF0900314E0FDAF77
:046F2C006C0261F59D
:107098007B017A037915E4FF126049900315E0300B
:0770A800E7037F00227F01D6
:0170AF0022BE
:107067007B017A037916E4FF126049900316E0303A
:08707700E704540FFF227F0023
:01707F0022EE
:107033007B017A037917126049900317E0FFF4602C
:0A70430007EF60047F0180027F0068
:01704D002220
:03718900202000C3
:0A6D5B00AB3FAA40A941121207FF46
:026D65008F4855
:106D6700E478ACF6E5481392927F0A7E00126778C2
:106D7700D2937F0A7E00126778C293E548C313F562
:0A6D87004878AC06E6C3940840DA31
:016D910022DF
:02648B008F6E12
:10648D00C293E4F58475D2FF75D30F7F0AFE1267B0
:10649D007875840F43A504AF6E126D6575840F5327
:1064AD00A5FBD2927F0A7E00126778E47879F61800
:1064BD00F6787A76013092077879E6797A47F6D2CE
:1064CD00937F0A7E00126778C2937F0A7E0012675F
:1064DD0078787AE625E0F6787806E6C3940840D514
:1064ED00E4F584F5D2F5D37F0AFE1267787879E664
:0164FD00FF9F
:0164FE00227B
:0659B5008B3F8A4089418E
:1059BB00C293E4F58475D2FF75D30F7F0AFE12678D
:1059CB007875840F43A5047FBF126D6575840F53E3
:1059DB00A5FBD2927F0A7E00126778E478A9F6E4E1
:1059EB0078AAF678A8F678AB760130920778AAE613
:1059FB0079AB47F6D2937F0A7E00126778C2937F0A
:105A0B000A7E0012677878ABE625E0F678A806E602
:105A1B00C3940840D578A9E6FFC39403501908E650
:105A2B00FEEFFDC374059DFDE49400AB3FAA40A9B6
:105A3B00418D82F583801E78A9E6FFC3940550182B
:105A4B0008E6FEEF7C0024FDF582EC34FFF583AB1A
:105A5B003FAA40A941EE801178A9E6B4060E08E6EC
:105A6B00AB3FAA40A94190000212124678A906E664
:105A7B00C3940750030259EAE4F584F5D2F5D37FBA
:055A8B000AFE0267782D
:106DFB008F468D47C293E4F58475D2FF75D30F7F11
:106E0B000AFE12677875840F43A504AF46126D65B1
:106E1B00AF47126D65E4F584F5D2F5D37F0AFE0218
:026E2B00677886
:106415008B3F8A408941C293E4F58475D2FF75D3D9
:106425000F7F0AFE12677875840F43A5047FBE129D
:106435006D65900005126D5B900004126D5BAB3FBE
:10644500AA40A941900003126D61AB3FAA40A94142
:106455001211EEFF126D65AB3FAA40A941900001F4
:10646500126D617F01126D65AB3FAA40A941900095
:1064750002126D61E4FF126D65E4F584F5D2F5D382
:066485007F0AFE026778A9
:106CE8008D6FEF14601614601914601C14601F1463
:106CF800602224057025AD6F7F86801CAD6F7F886C
:106D08008016AD6F7F8C8010AD6F7F84800AAD6F69
:0C6D18007F828004AD6F7F80126DFB2233
:10542D008B088A09890A1211EEFFF47049AB0BAA99
:10543D000CA90D900007743F121246900006743FA0
:10544D00121246900004743F121246900003743FEE
:10545D00121246900001743F121246743F1212341C
:10546D00AB0BAA0CA90D900005742D1212469000DD
:10547D0002742D02552AEFC4540F2430AB0BAA0C25
:10548D00A90D121234AB08AA09A90A1211EE540F74
:10549D002430AB0BAA0CA90D9000011212469000FE
:1054AD0002742D121246AB08AA09A90A9000011226
:1054BD001207C4540F2430AB0BAA0CA90D90000396
:1054CD00121246AB08AA09A90A900001121207543C
:1054DD000F2430AB0BAA0CA90D90000412124690AC
:1054ED000005742D121246AB08AA09A90A900002F4
:1054FD00121207C4540F2430AB0BAA0CA90D900047
:10550D0006121246AB08AA09A90A90000212120748
:10551D00540F2430AB0BAA0CA90D900007121246A4
:08552D00900008E4121246226E
:105318008B0E8A0F89101211EEF47049AB11AA1284
:10532800A913900007743F121246900006743F12AA
:105338001246900004743F121246900003743F1204
:105348001246900001743F121246743F121234AB99
:1053580011AA12A913900005743A1212469000027D
:10536800743A025422AB0EAA0FA91090000312122D
:1053780007C4540F2430AB11AA12A913121234AB6C
:105388000EAA0FA910900003121207540F2430AB75
:1053980011AA12A913900001121246900002743A41
:1053A800121246AB0EAA0FA910900004121207C4DD
:1053B800540F2430AB11AA12A913900003121246FD
:1053C800AB0EAA0FA910900004121207540F243034
:1053D800AB11AA12A913900004121246900005748A
:1053E8003A121246AB0EAA0FA91090000512120726
:1053F800C4540F2430AB11AA12A91390000612123C
:1054080046AB0EAA0FA910900005121207540F24DC
:1054180030AB11AA12A91390000712124690000887
:05542800E4121246220F
:106B24007B017A0279F61259B59002F6E0F4603FDF
:106B3400750B01750C02750DFC7B017A0279F61256
:106B4400542D7B017A0279FC126EDE7BFF7A717917
:106B540089126EDE7511017512027513FC7B017AC0
:0F6B64000279F61253187B017A0279FC126EDE69
:016B730022FF
:10712600E4FF12648B787BEFF6F460047F01800243
:027136007F00D8
:017138002234
:07717200E4FD7F8E026DFBBE
:100B8000020F41E86480F8E933E83360110460F053
:100B9000ED33EC337009E8FCE9FDEAFEEBFF2204DB
:100BA00060DED3EB9FEA9EE99DE8C2E78CF0C2F7D6
:100BB00095F0400CE8CCF8E9CDF9EACEFAEBCFFBA2
:100BC000120F0C85D0F05804700320D5B3E80470E0
:100BD000075002B2D5020F4B92D5EC0460F7E4CC7B
:100BE000C0E0C398F8603B94186008400DD0E0FB6B
:100BF000020F23E4FBFAC9FC8028E830E406E4C9CC
:100C0000FBE4CAFCE830E305E4C9CACBFCE85407BE
:100C10006010F8C3E913F9EA13FAEB13FBEC13FCC9
:100C2000D8F130F52FC3E49CFCEF9BFFEE9AFEED6C
:100C300099FDD0E0FBEF4E4D4C701222DB03020F0A
:100C400048EC2CFCEF33FFEE33FEED33FDED30E7E7
:100C5000EB020F23EF2BFFEE3AFEED39FDD0E0FB68
:100C600050130BBB0003020F4BED13FDEE13FEEF11
:080C700013FFEC13FC020F233B
:100C7800EC4D6011E8497017ED33EC3304600DE476
:100C8800FCFFFEFD22E933E8330470F8020F41123D
:100C98000F0C58046009E4CC24815006285009023E
:100CA8000F4B284003020F48C0E0EB4A7044B9805C
:100CB80006D0E0FB020F37EF4E701CBD8008EBFF3B
:100CC800EAFEE9FD80EBE98DF0A4FEE5F0020D6196
:100CD800E9CDF9EAFEEBFFEF89F0A4FCE5F0CE8957
:100CE800F0A42EFFE435F0CD89F0A42DFEE435F014
:100CF8008067EF4E7005BD80D780C3EF8BF0A4AC42
:100D0800F0EE8BF0A42CFCE435F0F8EF8AF0A42C7C
:100D1800E5F038FCE433CB8DF0A42CFCE5F03BF88F
:100D2800EE8AF0A42CFCE5F038F8E433CF89F0A47F
:100D38002CFCE5F038CF3400CE89F0A42FFFE5F085
:100D48003EFEE433C98DF0A42EFEE5F039CD8AF0DD
:100D5800A42FFFE5F03EFEE43DFD33D0E0FB500755
:100D68000BBB000F020F4BEC2CFCEF33FFEE33FEF6
:060D7800ED33FD020F2324
:100D7E00020F4BEC5D046005E859047003020F414D
:100D8E00120F0C580460F6EC4860F2EC7004FDFE95
:100D9E00FF22C860DB2481C85009C3986002500648
:100DAE00020F489850CAF582E9294B4A7005AB826A
:100DBE00020F3775F0007C1A7880C3EF9BEE9AED28
:100DCE0099400DC3EF9BFFEE9AFEED99FDE842F0C0
:100DDE00DC23ACF0D0E0FFD0E0FED0E0FDAB822013
:100DEE00E7101BEB60BAEC2CFCEF33FFEE33FEED9D
:100DFE0033FD020F23E803F830E705C0F075F0006D
:100E0E00EF2FFFEE33FEED33FD40B830E7C280AA80
:100E1E0074F8CC6480CCC86480C8F58204604FC37B
:100E2E00EB9FF5F0EA9E42F0E99D42F0E89C45F01A
:100E3E00603C501DE5825FFFE582D313CB5BCBF4A4
:100E4E002B5582FB50280ABA002409B900200880CD
:100E5E001DE5825BFBE582D313CF5FCFF4C3132F67
:100E6E005582FF50090EBE00050DBD00010CC3EBEF
:100E7E009FF5F0EA9E42F0E99D42F0E89C45F06055
:090E8E0007CC4820E701B3EC2277
:100E970075F020800E75F010800575F0087D007ED6
:100EA700007F003392D530D5031213A0EC334010E6
:100EB700EF33FFEE33FEED33FDEC33FCD5F0ED22DF
:0E0EC700E5F0247EA2D513CC92E7CDCEFF221B
:100ED500EDD2E7CD33EC3392D524814006E4FFFE15
:100EE500FDFC22FCE4CFCECDCC24E0501174FF8074
:100EF500EDC3CC13CCCD13CDCE13CECF13CF047011
:070F0500F030D5DE0213A05D
:102F5400E55D2449F8E6055D227846301C0278498F
:102F6400E475F0011214FC0211EE2015EB7F2ED251
:102F7400158018EF540F2490D43440D4FF30190B2B
:102F8400EF24BFB41A0050032461FFE55E6002150C
:102F94005E0561E56170020560301C0D7846E475DC
:102FA400F0011214FCEF0212340270B07403D21C4C
:102FB4008003E4C21CF55D8B468A478948E4F55ECC
:102FC400F560F561E55E60077F20122F8F80F5754F
:102FD4005FFFC216C215C217C218C21AC21BC21D95
:102FE400122F5DFF700D301C057F00122FA0AF6102
:102FF400AE6022B4255FC2D5C219122F5DFF24D062
:10300400B40A00501A75F00A785E30D50508B6FF88
:103014000106C6A426F620D5047002D21880D9244D
:10302400CFB41A00EF5004C2E5D21902328DD21681
:1030340080C6D21580C0D21780BCD2D580BAD21A2D
:1030440080B47F20122F8F2017077401B55E0040D3
:10305400F1122F54FF122F8F022FC8D21DD21B80C2
:1030640095122F54FB122F54FA122F54F94A4B7015
:103074000679847A337BFF20172EE55E602A7E0072
:103084008E8275830012120760060EEE655F70F083
:10309400C2D5EBC0E0EAC0E0E9C0E0EE1232EDD008
:1030A400E0F9D0E0FAD0E0FB1211EEFF60AAEBC029
:1030B400E0EAC0E0E9C0E0122F8FD0E02401F9D0AB
:1030C400E03400FAD0E0FBE55F0460DCD55FD98032
:1030D40087D21780A21232D060F7E55F7001041224
:1030E4000F56A95F600DE55F600914F55F12337731
:1030F400EF60F3EA30E702F404C3995077EAF42569
:103104005F0430E701E404F55F800D1232D060C142
:10311400EA055F255F120F56EA785CF630E701E4B2
:10312400255F04D55F04201A01141232EDE4C0E0D7
:10313400123377785CE6601320E70714F6122F77D2
:10314400802204F6D0E014C0E07F00122F77E55F00
:103154006007122F6E155F800B301A03122F6ED08A
:10316400E0022FC8D0E00480C51232D060A0E55F31
:1031740004120F56785CEAF6E55F201A0260010437
:0531840024041232EDED
:1031890074FF04C0E0123377122F77E55F201A022B
:103199006003122F6ED0E0B55FE87F45122F81786A
:1031A9005CE67F2B30E7047F2DF404C0E0122F8FFB
:1031B900D0E075F00A84C0F0122F78D0E0122F7891
:1031C900022FC8791080027908C21BC21D8008D25B
:1031D900D5790A8004790AC2D5E55F047002F55FE2
:1031E900E4FAFDFEFF122F54FC7B08201613122F60
:1031F90054FD7B1030150A122F54FE122F54FF7BF9
:1032090020EC3382D592D55013C3E43015069FFFC5
:10321900E49EFEE42016039DFDE49CFCE4CBF8C289
:1032290016EC700CCFCECDCCE824F8F870F38017EB
:10323900C3EF33FFEE33FEED33FDEC33FCEB33FB31
:10324900994002FB0FD8E9EB301605F8D0E0C448E5
:10325900B216C0E00AEC4D4E4F78207B0070C2EAEE
:10326900B55F0040BCC0E01232EFD0F0D0E02016CC
:1032790004C4C0E0C4B216C0F0122F78D0F0D5F063
:10328900EB022FC812153C30655331CC5830364CFF
:1032990030324231D04F31D84431D849304B4331A3
:1032A900DE55310F46316D4530D94733A450303A98
:1032B9002D303E2E30612B304223305F20338D2A52
:1032C9002FFA4800003059E55FB4FF03755F061215
:1032D9002F54FC122F54FD122F54FE122F54FF7835
:1032E90055020F85790AA2D5201814301A09B91088
:1032F900020404B9080104A2D5201B0250010420CC
:1033090017689217B55E005034C0E07F2030181955
:103319007F30A217721B721A500F123346C217C29E
:103329001BC21AC21D7F30800F301A03E9C0E01298
:103339002F8F301A03D0E0F9D0E0B55ECC301A17E0
:103349007F30B9100C122F8F7F583019077F788082
:1033590003B90803122F8F3017057F2D022F8F7F96
:1033690020201DF87F2B201BF322921780CF7F008E
:10337900B4070050052455F8E6FF22286E756C6CD9
:103389002900D216122F543016F8C216785E30D59D
:103399000108F6022FFA2D50434958122F542403DD
:1033A900B405004001E490339F93122F80743A12C0
:0A33B9002F80D218755E040231CC9B
:100F0C00E9D2E7C933E833F892D5EDD2E7CD33EC2B
:070F1C0033FC5002B2D522A4
:100F2300EC30E7100FBF000C0EBE00080DBD00042F
:100F33000BEB6014A2D5EB13FCED92E7FD2274FFDB
:100F4300FCFDFEFF22E480F8A2D574FF13FC7D8034
:030F5300E480EF48
:100F5600F920E72824F950037907E4F42402FB1862
:100F6600DBFDE624FB5014E9600DE4F618E604F612
:0F0F7600B40A08E4F6D9F57401F60A22C2D522AE
:100F8500ED33EC3392D5FA602AB4FF33EDC2E77B3B
:100F9500FF60067A0F79AAE4227A0F79B320D50487
:100FA5007A0F79AE224E614E002B494E46002D49EF
:100FB5004E4600E47A08F608DAFC7B00740722E85E
:100FC500C0E0ECC0E0EDC0E0EEC0E0EFC0E0EA75E7
:100FD500F010A4CAABF075F04DA42BFBE435F0FC82
:100FE500EA2410FAEB34C5FBEC34D9FCEDC2E7FF7B
:100FF50075F056A4F42411C5F0F434C58FF0A42A75
:10100500E5F03BE43CF620E7141210B8D0E0FFD041
:10101500E0FED0E0FDD0E0FC120D818014F4041256
:1010250010B8D0E0FFD0E0FED0E0FDD0E0FC120C1F
:1010350078D0E0F8E6FAEDD2E7CD33EC332482FB45
:10104500E4C3CF33CFCE33CECD33CD33DBF37B0704
:1010550075F00A846004F6081B0AE5F0F6088FF0BF
:10106500740AA4FFACF08EF0740AA42CFEACF05008
:10107500010C8DF0740AA42CFDE435F0F608DBDED6
:03108500740722CB
:101088003F8000004120000042C80000447A000070
:10109800461C400047C35000497424004B189680F2
:1010A8004CBEBC205A0E1BCA6753C21C749DC5AEE9
:1010B800FB60065407601C23231210E6EB543860CB
:1010C800091210D21210E1120C78ECF8EDF9EEFAD0
:1010D800EFCB22EB1210E180F1543803241C90105E
:1010E80088FE93FC0EEE93FD0EEE930ECE93FF2238
:0300000002616535
:0C616500787FE4F6D8FD7581B20261ACD1
:1010F800E709F608DFFA8046E709F208DFFA803EDA
:1011080088828C83E709F0A3DFFA8032E309F608C6
:10111800DFFA8078E309F208DFFA807088828C832E
:10112800E309F0A3DFFA806489828A83E0A3F608E2
:10113800DFFA805889828A83E0A3F208DFFA804CBC
:1011480080D280FA80C680D4806980F28033801093
:1011580080A680EA809A80A880DA80E280CA8033FC
:1011680089828A83ECFAE493A3C8C582C8CCC58374
:10117800CCF0A3C8C582C8CCC583CCDFE9DEE78044
:101188000D89828A83E493A3F608DFF9ECFAA9F0C3
:10119800EDFB2289828A83ECFAE0A3C8C582C8CC19
:1011A800C583CCF0A3C8C582C8CCC583CCDFEADE32
:1011B800E880DB89828A83E493A3F208DFF980CC94
:1011C80088F0EF60010E4E60C388F0ED2402B4048D
:1011D8000050B9F582EB2402B4040050AF23234534
:0611E80082239011487300
:1011EE00BB010689828A83E0225002E722BBFE02FF
:0911FE00E32289828A83E4932232
:10120700BB010CE58229F582E5833AF583E022509C
:1012170006E92582F8E622BBFE06E92582F8E222E6
:0D122700E58229F582E5833AF583E4932200
:10123400BB010689828A83F0225002F722BBFE0199
:02124400F32293
:10124600F8BB010DE58229F582E5833AF583E8F0DE
:10125600225006E92582C8F622BBFE05E92582C88A
:02126600F22272
:10126800EF8DF0A4A8F0CF8CF0A428CE8DF0A42E9A
:02127800FE2254
:10127A00BC000BBE0029EF8DF084FFADF022E4CC58
:10128A00F875F008EF2FFFEE33FEEC33FCEE9DEC21
:10129A00984005FCEE9DFE0FD5F0E9E4CEFD22ED67
:1012AA00F8F5F0EE8420D21CFEADF075F008EF2FB1
:1012BA00FFED33FD4007985006D5F0F222C398FDA2
:0512CA000FD5F0EA223F
:1012CF00C2D5EC30E709B2D5E4C39DFDE49CFCEE3A
:1012DF0030E715B2D5E4C39FFFE49EFE12127AC326
:1012EF00E49DFDE49CFC800312127A30D507C3E421
:0612FF009FFFE49EFE22A9
:10130500BB010A89828A83E0F5F0A3E022500687B3
:10131500F009E71922BBFE07E3F5F009E319228975
:0B132500828A83E493F5F074019322A8
:10133000BB0110E58229F582E5833AF583E0F5F0FB
:10134000A3E0225009E92582F886F008E622BBFED8
:101350000AE92582F8E2F5F008E222E5832AF5831E
:08136000E993F5F0A3E99322E3
:10136800BB010789828A8302158E500B09C5F027B5
:10137800F7C5F01937F722BBFE0D09F8E325F0F39E
:10138800C5F019E338F322F889828A83740193251A
:08139800F0C5F0F8E4933822DF
:0E13A000C3E49FFFE49EFEE49DFDE49CFC225E
:1013AE00EB9FF5F0EA9E42F0E99D42F0EC6480C8B6
:0613BE0064809845F02256
:1013C400EB9FF5F0EA9E42F0E99D42F0E89C45F07F
:0113D40022F6
:1013D500E8600FECC313FCED13FDEE13FEEF13FFF6
:0313E500D8F1221A
:1013E800BB010789828A8302145E5005E9F802145A
:1013F80052BBFE05E9F80215A489828A830215B05A
:10140800BB010DE58229F582E5833AF58302145E76
:101418005007E92582F8021452BBFE07E92582F835
:101428000215A4E58229F582E5833AF5830215B011
:10143800BB010789828A830214BF5005E9F80214A8
:0A144800B3BBFE05E9F80215DD2232
:0C145200E6FC08E6FD08E6FE08E6FF22C6
:0C145E00E0FCA3E0FDA3E0FEA3E0FF2201
:0D146A00E6FB08E6F908E6FA08E6CBF822F2
:0C147700E0F8A3E0F9A3E0FAA3E0FB22F8
:10148300BB010DE58229F582E5833AF583021477E2
:101493005007E92582F802146ABBFE07E92582F8A2
:1014A3000215C0E58229F582E5833AF5830215CD5D
:0C14B300ECF608EDF608EEF608EFF62265
:0C14BF00ECF0A3EDF0A3EEF0A3EFF022A0
:1014CB00A8828583F0D083D0821214E21214E21228
:1014DB0014E21214E2E473E493A3C583C5F0C5834D
:1014EB00C8C582C8F0A3C583C5F0C583C8C582C86B
:0114FB0022CE
:1014FC00FAE6FB0808E6F925F0F618E6CA3AF622F1
:10150C00BB010DE58229F582E5833AF5830215F2DC
:10151C005007E92582F80215E9BBFE07E92582F898
:10152C000215FBE58229F582E5833AF58302160460
:10153C00D083D082F8E4937012740193700DA3A33E
:10154C0093F8740193F5828883E473740293686052
:06155C00EFA3A3A380DF52
:106EDE001211EE601CFF09E970010AC0E0EAC0E081
:106EEE00EBC0E01270B0D0E0FBD0E0FAD0E0F98059
:0A6EFE00DF7F0A1270B0E4FEFF22ED
:106828008B468A4789488B4C8A4D894EAB4605482A
:10683800E548AA477002054714F91211EE70ED7485
:10684800FF2548F54874FF3547F547AB49054BE543
:106858004BAA4A7002054A14F91211EEFFAB46051D
:1068680048E548AA477002054714F9EF1212347038
:08687800DAAB4CAA4DA94E2237
:106A30008B468A478948E4F54EF54FE54D154DAE36
:106A40004C7002154C4E6033AB49AA4AA94B121147
:106A5000EEFFAB46AA47A948054FE54FAC4E700282
:106A6000054E14F5828C83EF121246EF60CD74014F
:106A7000254BF54BE4354AF54A80C0AB46AA47A9F9
:026A80004822AA
:10000E00E4FFFE1211EE600C0FEF70010E09E970A5
:05001E00F20A80EF2250
:10701700E94A4B7001221211EEFF6D700122EF70E9
:0C70270004FBFAF92209E970ED0A80EA86
:1069DA008B478A4889498B4A8A4B894CAB4AAA4BCE
:1069EA00A94C1211EE600D7401254CF54CE4354B9F
:1069FA00F54B80E8AB4AAA4BA94C1211EE6D700117
:106A0A0022E54C154CAA4B7002154BF9E54785480F
:106A1A0083854982654A7008E965827003EA65835D
:066A2A0070D2FBFAF92214
:10156200EF4E6012EF60010EEDBB010B89828A83A0
:10157200F0A3DFFCDEFA2289F05007F709DFFCA9AD
:0C158200F022BBFEFCF309DFFCA9F02204
:10617100027080E493A3F8E493A34003F68001F254
:1061810008DFF48029E493A3F85407240CC8C3332F
:10619100C4540F4420C8834004F456800146F6DFFE
:1061A100E4800B01020408102040809068D7E47E4F
:1061B100019360BCA3FF543F30E509541FFEE493F3
:1061C100A360010ECF54C025E060A840B8E493A3BA
:1061D100FAE493A3F8E493A3C8C582C8CAC583CAE5
:1061E100F0A3C8C582C8CAC583CADFE9DEE780BE9D
:01692D000069
:10158E00C5F0F8A3E028F0C5F0F8E58215827002E8
:06159E001583E038F02285
:0C15A400E2FC08E2FD08E2FE08E2FF2283
:1015B000E493FC740193FD740293FE740393FF2281
:0D15C000E2FB08E2F908E2FA08E2CBF822AB
:1015CD00E493F8740193F9740293FA740393FB2274
:0C15DD00ECF208EDF208EEF208EFF2224A
:0915E900E6FB08E6FA08E6F92227
:0915F200E0FBA3E0FAA3E0F922FA
:0915FB00E2FB08E2FA08E2F92221
:0C160400E493FB740193FA740293F92242
:00000001FF
